:020000041100E9
:10300000002373B52B4D2C4C28006361022601F080
:1030100061F94021FE2221742800284B009601F01E
:10302000ABF9002836D1217CFF222800244B0096E2
:1030300001F0A2F900282DD1224BA2899A4226D173
:10304000E389214A93420DD1204B6361204B2268D2
:10305000002A03D1002B01D043CB43C4280001F048
:1030600077F973BD1B4A934201D00023EFE71A4B57
:103070001A4A1B68934206D9C02304222800217CE7
:103080009B0001F0EFF9114B6361154BDFE7002363
:103090002374EAE7CC233821AC2228009B01217459
:1030A00001F0E0F90028F2D10E4B63610E4BE38191
:1030B0000E4BCCE7643CFF1FFC5BFF1F085CFF1F4F
:1030C0000A5CFF1F595900008305000001410011EF
:1030D000C4B8001182150000205CFF1F8713000098
:1030E000D0B80011B9410011AAAAFFFFB8B8001169
:1030F000F7B5164B0192C318021D002000938823D8
:103100005B05D3181B685C1C1AD09CB2402C18D8E5
:103110008D781E0CAC466746CD782D023D43AE42FD
:1031200006D1019800280ED110000C70240A4C70B2
:1031300003249BB20733A343D218009B9A42DED3E9
:10314000FEBD4432F9E71000FAE7C046FC0F00006C
:10315000802213B503000324019189B25201073183
:103160009B18A14304305A1A88235B05C3181B68B7
:10317000591C03D190429241104016BD99B240298A
:1031800007D80B000733A343C0189042ECD30020AC
:10319000F3E74430F9E7134B134A1B68126810B584
:1031A000FA24934201D81A00F824104BE4021B6859
:1031B0009A4210D813000E4A12689A420ED3013375
:1031C00007D1F823DB029C4203D10A49054808F0E5
:1031D000D7FA200010BDFC24E402ECE7FE24E40250
:1031E000F7E7C04600C0071100D0071100E0071143
:1031F00000F00711FFFFFF7FF0B59BB015000490B2
:103200000391402A00D9A0E006AB59801A80FFF74D
:10321000C2FF0400042816D9002206A9FFF768FFA0
:10322000052810D906AB1B88AB420CD1002D07D066
:10323000514B2A000499C01808F06AF9002802D1FD
:1032400001201BB0F0BD06AB1D8020000699FFF7E2
:103250007FFF041E7BD1069B0793FFF79CFF802313
:103260005B01C618802307001B039E4201D3F8268A
:10327000F60288235B05F31801931B68013302D023
:10328000019808F09DF83D49019808F079FA3B1D36
:103290000293331D05938822029B52059B181B68DD
:1032A00008935A1C3CD044219AB20091402A04D879
:1032B0000320D11D814389B2009103991B0C8B42DD
:1032C00024D0402A22D80122300008A9FFF710FF9D
:1032D000021E1BD1380008A9FFF70AFF04000428CA
:1032E00031D9009A059B9B1880225201B218934253
:1032F00040D288235B05C118009A09A808F028FA73
:103300001D4B009A09A9F01808F08AF8009A029B50
:103310009446634402931A4B029AFB189A42BAD31A
:1033200088235B05FC1821680198013908F028FA08
:10333000200008F045F8039A07AB5A80300007993F
:10334000FFF706FF0400002C03D1002079E70428D2
:10335000FBD988235B05E018069908F011FA0323CE
:10336000EA1C9A4300D16BE7034B0499E01808F07C
:1033700057F865E70424ECE704000011FFFFFF7F26
:10338000F80F0000F7B505001400402A21D80027E7
:1033900001AE71803780FFF7FEFE042816D93A008F
:1033A0003100FFF7A5FE042810D93688BC420BD0A7
:1033B000BD4209D0221CB44200D9321C064B92B245
:1033C000C118280008F0C4F930B2FEBDC04300B2F5
:1033D000FBE703204042F8E70400001137B5042260
:1033E00004000D0001A81649FFF7CCFF02000428D5
:1033F0000BD1019BA34208D3AB4204D0104901A8D2
:103400000195FFF7F9FE01203EBD0E4C2368200018
:10341000019307F0D5FF019920000139019108F0CF
:10342000AFF980235B01E418074B9C42EED10422E4
:10343000034901A80195FFF7DFFE0020E4E7C0463D
:103440005555000000C007110000081130B589B0C3
:1034500008F0DEF810226946254807F0E9FE254B02
:10346000009A9A420ED1019B029A0F2B33D8002169
:1034700001240698013B08D2002900D00292029B49
:10348000013331D10023029325E0551CF2D1020013
:103490002100EFE710341022200004A907F0C8FE35
:1034A000029B013301D1069B0293882304995B059B
:1034B000C918059B06981A03120B049105928142C4
:1034C00003D02B4201D108F043F9019B013B01934A
:1034D000019B002BDED1029B002B03D004930498A8
:1034E0004168084709B030BDE025014C2D03EFE7E6
:1034F00000000111504859368022F8B5964C974B80
:10350000D200002120001C6007F0FAFE2300944A3C
:1035100088331A60934B1A786A23002A00D011333B
:10352000E3620A232365904B37221B780821A363AB
:103530008E4B6018E361102323628D4B3B25636142
:10354000C823DB00A36123008C331A602823013ACF
:10355000E26321646364C267043A201DC2672000ED
:10356000BC3005602000C03001602000C430036022
:1035700020000635CC3005602000083DC8300560CD
:103580002000D03002602200D43211602200D832F4
:10359000136022000226E032200016604222DC3056
:1035A000026020001B3DE43005602000E83001602F
:1035B0002000EC30036023000520F4331860230062
:1035C000F0331A602300183290331A6023009433CA
:1035D000196023001E3A98331A60AF23DB00236082
:1035E000644BFA252363644B6448A3642300B93217
:1035F000FC33FF32AD00A260E56022611D60A06275
:103600007320E0656D386065A065FA2796203F015C
:103610008000E76465625960A0660920E0660020CA
:10362000616757496666E167564E57492667A06746
:103630000F601527676027001A219C373960270023
:103640000731A037396027004B49A837396021007E
:10365000F8310D6021006427A4310F6021005F3F25
:10366000AC310F602100033FB0310F602700B43749
:103670003D00C8272F6027003825B83738609D6087
:10368000424D96215D64424D8900DD61414D1962D4
:103690005D62F53DFF3D9D621E253949DD66596637
:1036A000996499673C49DE651E6618675867D96753
:1036B000BE233A495B00E1508130394BFF30235043
:1036C00004302150C42149006350C623E4205B002C
:1036D000E2500433E2503349334A344BD160344929
:1036E000800019503349E938FF3819503249043005
:1036F000195032493248D16132491163324951631C
:103700001900F4310860CE20304940001160304982
:10371000195019002F48F83108602F49D1658221CE
:103720002E4A89005A501A002D490832D1671A00D2
:103730002C49B432116088212B4A89005A501A0052
:103740002A49883211602A4ADA6407F031FD0120E3
:1037500007F06EFFF8BDC0460004FF1F985EFF1F14
:103760007069FF1F903EFF1F4A0AFF1F3A070000C3
:1037700080C3C9019A02000050C300006A1800000B
:1037800088130000204E0000F009FF1F6509FF1F8D
:1037900068100000C4090000DC05000040420F0072
:1037A00010270000D91AFF1FFC00FF1F0000FF1F99
:1037B0008127FF1FC52AFF1F5D29FF1F251EFF1F31
:1037C0007523FF1F411EFF1FED1FFF1FB11DFF1FB0
:1037D0000124FF1FE924FF1FD918FF1FB923FF1F72
:1037E000C921FF1FD521FF1FB11CFF1F691DFF1F2E
:1037F0009D1CFF1F0223F0B501245E4D5E4E2B7011
:103800005E4B91B01C705E4F03933368002104201F
:10381000BB7006F0DFFB042006F0D6FA00239842C6
:1038200005D0BA78552A02D0332A00D096E033600A
:1038300007F0A6FEFFF760FE1F2201240021514B76
:1038400010AE1A70504B1C70504B1970504B1968C9
:103850009143163A0A431A60602219689143403A2C
:103860000A431A6007F0DCFC07F0A2FEC120FF212A
:10387000484B80001A588A431A50C5229200985823
:103880008843BF39014399509858434908408021E3
:10389000C9010143802099509958C0050902090ABD
:1038A0000143995080213D48490107F099FE0323C7
:1038B00022003B49019400933A4807F0F9FC2C227E
:1038C000394905A807F044FF05AC61782078023437
:1038D00006F09AFAA642F8D1344C1120002106F0E5
:1038E000A7FB2268324B03201A40A023DB021343BC
:1038F0002360802322689B041343236022682D4B9E
:103900001A4080239B03134323602B4A2B4B934283
:1039100000D8012007F0ECFC07F052FE802322685B
:10392000DB0413432360287807F0CAFD039B187853
:10393000C0B207F0DDFE07F09BFC2149042007F030
:1039400017FE06F08DFC00F0A7F800F0B7FD00F0C0
:103950005FFE00F003FA002011B0F0BD00932100DB
:10396000174A042007F06CFE8023DB059C62FFF7FA
:103970006DFD5DE74A0AFF1F34F00040903EFF1FD7
:103980002C5CFF1F480AFF1F490AFF1F680AFF1F20
:10399000BCF0004000E100E0FF00FFFF943EFF1F8D
:1039A0001851FF1F944EFF1FE0B7001114F00040A4
:1039B000FF7FF8FFFFFF9FFF0080FF1F7069FF1F61
:1039C0003B00010870B500252549264A26484D636D
:1039D00008CA1B051B0DED188242F9D10026802272
:1039E000224B92058B630921214B224C1E62224BF4
:1039F0001120DA67214BDA688A43DA609A68204935
:103A00000A409A60266007F0C3FC112007F040FDD1
:103A10008022636C93436364EE24E4006C43194A90
:103A2000200C0400642390420AD8FA223300D2000A
:103A3000904205D9144B0A21C01807F0F9FCC3B213
:103A4000124A11201372D48007F03AFC104B1B78F5
:103A5000002B04D10F4B1021187807F0F9FC70BD32
:103A6000000005408805054000060540FF010000F4
:103A700000F000400038004004E100E03CF000406D
:103A8000FFDFFFFFB70B000030F8FFFF145CFF1FE4
:103A90004E5EFF1F4C5CFF1F002210B5110011206D
:103AA00007F0DEFB10BD0000002370B50925334E82
:103AB000334C3362E3681120AB43E36007F0E8FC6A
:103AC000112007F065FC112007F0E2FB402322687B
:103AD00011201343236080236268DB021343636079
:103AE0008023A2681343A360A368264A1340A360FF
:103AF0008023A2689B0113431022A360236C93438D
:103B000023640123226C1A43226480225200326211
:103B1000216B1D4A11402163616B11406163A16BF0
:103B20001140A163E16B0A40E263E26817490A4071
:103B3000E260174A11680B43136007F0E9FDFD21AD
:103B4000144B154A89005A508023C720626B5B03CF
:103B500013436363E36880001D43104BE56019580D
:103B60000F4A1140802212020A431A508022920505
:103B70001A6008220B4B5A6370BDC04600F000402B
:103B80003CF00040FFFFDFFFEFFFEFFFFFFF7FFF95
:103B9000003800400000FF1FC539001100E100E0BF
:103BA000FF00FFFF0000054030B503A804880B208C
:103BB000002C0ED14968074D087849780902014365
:103BC0000A20A94205D1012120001980024B1B7A4D
:103BD000137030BD192A0000145CFF1FF7B51500E3
:103BE00008AA16884A680F4F1478527812022243A6
:103BF0000A24BA4214D10122DBB2019200962A00B3
:103C000007F068FA041E0BD1074B1B68002B07D086
:103C100068782A78000210434242504101309847A8
:103C20002000FEBD02290000985BFF1F30B5012572
:103C300003790400BFB02B4211D00A49408806F036
:103C4000B5FD28420BD0084B01A95B8D4D800B8040
:103C5000064B00221B7A60880B7103F09DFE3FB07B
:103C600030BDC046905BFF1FD83AFF1F145CFF1F9A
:103C700010B50549054806F04FFD0421044A0548E2
:103C800006F00CFD10BDC046905BFF1FFFFF00005B
:103C90000CB80011D83AFF1F10B5024804F0FEFC22
:103CA00010BDC0462D3C0011062310B583701033A3
:103CB0000371443B43712A3383714433C37100233E
:103CC0000222012103720E4B027041701C88817226
:103CD0004472197A0273C1729A784273DA788273E5
:103CE0000322C2731A7902745A7942740C228274C4
:103CF0009A79C274DB7903751123C370152010BD46
:103D0000145CFF1F10B5142007F08AFC124B14221C
:103D10000021186007F0F4FA002007F0F9FA0120FA
:103D200007F04EFA022007F063FC032003F05AFF6D
:103D3000042005F06FFF052003F098F9062003F03A
:103D400065FE072001F0FCF9082006F087FC092039
:103D500000F0E6FF10BDC0469C5BFF1F07F008FBAC
:103D6000012007F0F5FB07F0BBFC0000094B10B584
:103D70000400984205D0012904D12000064906F02C
:103D8000CBFC10BD0229FCD1013904F045FC002810
:103D9000F3D0F6E7FEFF0000C25BFF1F70B50D7A9F
:103DA000100004AA2C00168810221440154220D1BD
:103DB000002E20D10A78022A18D14A685178157845
:103DC0000E4A09022943914205D00D4A914209D079
:103DD0001C800A2404E014220A491A8007F0B8FC67
:103DE000200070BD0C2208491A80F7E71C800124CE
:103DF000F6E70824F4E70B24F2E7C046F3FF0000DF
:103E0000F4FF0000203DFF1FE8B8001110B50400CA
:103E10000749084806F080FC074804F07FFB0020B3
:103E2000E40704D50721054A054806F037FC10BD14
:103E3000C25BFF1FFFFF00006D3D001150B8001175
:103E40001C3BFF1F00B50C4BBFB01A780B4902A8F2
:103E500000F098FC6B4680B2D880002809D06A46F2
:103E6000074B01A91B889380064B0022188803F09A
:103E700093FD3FB000BDC046A05BFF1FA15BFF1FCD
:103E8000763BFF1F803CFF1F00B50C4BBFB01A787C
:103E90000B4902A801F0C6FC6B4680B2D88000280E
:103EA00009D06A46074B01A95B8D9380064B00221F
:103EB000188803F071FD3FB000BDC046CA5BFF1F0C
:103EC000CB5BFF1F1C3BFF1F803CFF1FF7B50E00A5
:103ED000377A1C0008AB11003D001A8820231D40D2
:103EE0001F423CD13378022B3BD173681F785B783B
:103EF0001B023B431E4FBB4208D01E4FBB4214D097
:103F00001D4DAB4221D00A252800FEBD002A2AD132
:103F1000142C2AD82200F06807F01AFC174B1C70EA
:103F2000012CF1D9FFF7B0FFEEE7002A1BD1202CBE
:103F30001BD82200F06807F00BFC114B04211C7009
:103F4000104B187807F084FADEE7E3B20124009200
:103F500001940A00310007F0BDF80500D4E70825F8
:103F6000D2E70125D0E70B25CEE70D25CCE7C046EB
:103F7000F3FF0000F4FF000002290000CA5BFF1FEE
:103F8000A05BFF1F4C5CFF1F332310B504000370C0
:103F90000A220749013007F0DBFB064B0F201B68A4
:103FA0001A0AE37222731A0C1B0E6273A37310BDFC
:103FB000145CFF1F3C5CFF1F30B501250379040032
:103FC000BFB02B4213D00B49408806F0EFFB2842CC
:103FD0000DD06A46084B02A81B889380FFF7D4FFD8
:103FE0006B46D8800022608801A903F0D5FC3FB061
:103FF00030BDC046C25BFF1F763BFF1F10B50248B5
:1040000004F04CFB10BDC046B93F001170B516005E
:1040100004AA148805AA15784A6850781178000215
:104020002A4A0843801805284BD807F021FA0313C1
:104030001E29343F0720032C0BD80422121BAA424E
:1040400000D92A0022491A803000091907F080FBA4
:10405000002070BD0720112CFBD81222121BAA428F
:1040600000D92A001B491A80EEE707200E2CF0D851
:104070000F22121BAA4200D92A0017491A80E3E72F
:104080000720032CE5D80422121BAA4200D92A00DB
:1040900012491A80D8E70720032CDAD80422121B11
:1040A000AA4200D92A000E491A80CDE70720032C26
:1040B000CFD80422121BAA4200D92A0009491A802B
:1040C000C2E700220A201A80C3E7C046DCD5FFFF02
:1040D0009BB80011E85BFF1F8BB8001186B8001178
:1040E00081B800117CB8001110B50D21024A0348B7
:1040F00006F0D4FA10BDC04670B800118C3BFF1F0B
:10410000F0B50024274E85B03000B47100F0E2F81D
:10411000254D264BEA89297C9A422FD10423300071
:1041200003AA00F057F90400300000F011F9012350
:10413000B371002C34D16B4699892B68C9BA4B43B3
:1041400029891B4A1B145B1853806B46D9896B68FD
:1041500049BA89B24B4369891B0C5B181548191C75
:104160001BB2834200DD011C0B0400D50021138823
:10417000918001331380200005B0F0BD022722009A
:1041800003AB3000009700F0F7F80E230400297C01
:104190000122300000976B4400F0EEF80443C3E7BF
:1041A0001C00E8E7643CFF1FFC5BFF1F8305000069
:1041B000145CFF1F0F27000073B5234E300000F082
:1041C00089F8224D07236A463000297C00F002F965
:1041D00004003000002C33D16B461B787F2B2FD886
:1041E00000F0B6F86B46D878F02302041B031A409F
:1041F0006B469B8816495BBA9BB21A432B68000931
:1042000053432A891B0C9B184B806B465A789B782A
:1042100012031B011A436B68024353436A891B0C48
:104220009B180C481A1C1BB2834200DD021C1304AD
:1042300000D500220B888A8001330B80200076BDD8
:1042400000F086F80124F9E7643CFF1FFC5BFF1FC8
:10425000145CFF1F0F27000070B5114C237C002B4E
:104260000FD0382B0ED10F4D280000F033F8CC239F
:10427000AC222800217C9B0100F0F4F8280000F01B
:1042800067F870BD084BE2899A42FAD1054D2800C3
:1042900000F020F800222800217C00F0C5F8EDE7AE
:1042A000FC5BFF1F643CFF1F8305000010B5084B3B
:1042B0001A7C002A09D05B69002B06D09847041E9F
:1042C00001D0FEF79DFE200010BD0124F9E7C04695
:1042D000FC5BFF1F70B5C17905000C00631E9C419B
:1042E0001A4BE402E41849000460C9B2007905F0F1
:1042F000D5FEE979687949000131C9B205F0CEFEF1
:10430000E8790930C0B206F0C3FF0023E3666133E9
:104310002360AA795B3B002A0ED022689A43023BB5
:10432000134323600A23E3610733236200232363DB
:10433000A3630133E36370BD22689A4302231343EE
:104340002360462363610633A361EFE7005000401A
:1043500070B5002504000368DD66C0790930C0B27D
:1043600007F096F82900207905F034FE29006079DD
:1043700005F030FE70BD0000F8B51E0006AB1D78DC
:10438000002304681700E366616007F041F9012328
:104390008022E3662B0027615200013B08D206F021
:1043A00027FF08200A4A1168002D03D12800F8BD14
:1043B0002261F2E7236F034203D02369013D33708A
:1043C000013613685B1A032BEED90125EEE7C046D0
:1043D0006008FF1F70B51C00002305681600EB661F
:1043E000696007F015F901238022EB662300520073
:1043F000013B08D206F0FCFE08200A4A1168002C96
:1044000003D1200070BD2A61F2E72B6F034203D075
:104410002B69013C3370013613685B1A032BEED90C
:104420000124EEE76008FF1F002370B50468150043
:10443000E366616007F0ECF80123E366256106F0AE
:10444000D7FE8020064A80001168636B034205D1C5
:1044500013685B1A032BF8D9012070BD0020FCE71C
:104460006008FF1F70B51D00002304681600E36696
:10447000616007F0CDF80123E36626610F33626BBC
:104480001A42FCD02B0A23611023626B1A42FCD023
:10449000EDB2256106F0ACFE8020074A800011686D
:1044A000636B034205D113685B1A032BF8D9012013
:1044B00070BD0020FCE7C0466008FF1F10B5084C27
:1044C000E368002B08D18022064B52021B689B1820
:1044D0006360054B1B68236007F062F8A06010BDA5
:1044E0003C5CFF1FC8F00040CCF0004070B5184A9B
:1044F000936A916A9942FBD116498A689A421FD3FE
:104500009A1A8B60144B0126186893B2D202D20E0D
:104510004343424300204C681B0A1B1912029B189C
:104520000E4C0A684B60551CA3420CD8002801D0E1
:104530004B600A600A4A136008680A4B186070BD35
:10454000581E821ADDE7084A30009B182A00EAE765
:1045500000F000403C5CFF1F140AFF1F40420F00A8
:10456000C8F00040CCF00040C0BDF0FF70B51F4C5B
:1045700023793F2B01D93F2323711D4B22791A70D8
:104580001878C0B207F094F818231A491A4A0B8019
:104590001A4913800B805380A379194980200B801E
:1045A0000C21938001334B43164D191C00018342AB
:1045B00000D9011C2980D1806379002B11D10133EE
:1045C0006371237A012B01D8022323726279237A43
:1045D0000D4853430A21584306F02AFF0B4D28602B
:1045E00070BDA02BEDD9A023EAE7C046305CFF1FC9
:1045F000480AFF1F7E3CFF1F3C3EFF1F7C3CFF1F05
:104600007A3CFF1F783CFF1F71020000205CFF1FF7
:10461000F8B514210020FEF7E1FE114C011E114DEA
:1046200009D10C22104BC1CBC1C4280006F068FE92
:10463000FFF79CFFF8BD0C2220000C49FEF7A2FEFC
:104640000C2802D0084B43CB43C40C222800084955
:10465000FEF798FE0C28EBD00C220021E5E7C046BF
:10466000305CFF1FFC5BFF1FDCB80011FC0C00007E
:10467000F50C0000F0B51D4C8022A54404008820F4
:1046800069465201400506F08BFD902212016A44F2
:104690001300200032C832C316C816C38023144C3E
:1046A000144FA6689B033343A3603B6006F070FF82
:1046B0008823A0685B05C01806F082FE00258823C9
:1046C00029008022A0685B05C01840196944520087
:1046D00006F0A6FE80230135FF355B019D42EED139
:1046E000A6603E60044B9D44F0BDC046FCEFFFFF5A
:1046F000B03DFF1F9808FF1F04100000F0B5040034
:1047000087B0002825D0684606F0CAFD1B4C022859
:1047100006D106226946200006F0FAFE002816D0CF
:104720006946002301250F262F00E25C01331009A2
:104730001030874038002F00324097403A00024343
:104740004A610439062BEFD16846FFF793FF07B0A3
:10475000F0BD182269460A4806F022FD6A46A30009
:10476000D358013305D01822FF21684606F0C8FD52
:10477000EAE70134062CF1D1E9E7C0466509FF1FDD
:1047800000090011F0B5002504000E0085B0AA4212
:1047900000D183E04B1C087801934B7889783779F6
:1047A00009021943F3783F061B040B431F43039789
:1047B00020706570252800D193E033D8112813D8D4
:1047C00006F0BEFE66000D010D010D010D01A700F2
:1047D000B500AE000D010D010D010D010D010D0122
:1047E0000D010D01E7000701232800D1C0E0DB28FF
:1047F00000D016E1042A00D8A9E01025052A05D02A
:10480000551F2A003800711D06F0A2FF0522310055
:10481000200006F09DFF2A003900601D06F098FF79
:1048200005353BE0562856D010D8332800D19AE001
:10483000552836D02628DAD1894B290013221800B2
:104840001D0006F05DFDFEF7DBFB59E0712800D18D
:1048500074E0722800D17DE0DC28C8D1022A00D89B
:1048600075E07378BFB26370B378A370032A05D084
:10487000033A390092B2F01CFEF7BEFC1022390058
:10488000E01CFEF77FFDC51C002807DA60705CE0C5
:104890000C222000734906F05BFF0C25280005B0B0
:1048A000F0BD013A704D0C2A13D8002A0AD0280016
:1048B000019906F04DFFFFF759FE0C2228006B49C5
:1048C000FEF79AFC29000C22601C06F041FF0D2522
:1048D000E4E70C22EBE7644D654B2A0043CB43C26F
:1048E000E9E7013A5E4D0C2A11D8002A08D0019957
:1048F000280006F02DFF0C2228005E49FEF77CFC04
:1049000029001322601C06F023FF1425C6E70C22A1
:10491000EDE705225849601C06F01AFF0625BDE7A1
:1049200012225649601C06F013FF1325B6E7082231
:104930005349601C06F00CFF0925AFE77178F02998
:1049400005D8504B188801F0C9FB0225A6E7FF23C4
:104950006370FAE74C4B012A03D072785A70627088
:10496000F3E75B78F4E72000FFF70EFB050095E71F
:10497000042A04D9454D2F6006F012FEA860FFF707
:10498000B5FD0422039003A9601C06F0E1FE052595
:1049900084E73F4D062A15D906222800019906F022
:1049A000B7FD00280ED006220199280006F0D0FE9F
:1049B000062238492800FEF71FFC0123324A5178AD
:1049C0000B43537029000622601C06F0C1FE072528
:1049D00064E7012ABBD07078FFF790FEB5E70128A5
:1049E00000D004E7931E2C4F1A2B04D87378002BA9
:1049F00009D100F009F9294B39001D78601C6A1EA5
:104A000006F0A6FE4AE7551E2A000199380006F076
:104A10009FFE2349AAB23800FEF7EEFB00F02AF908
:104A2000E9E7DA2893D1042A91D9082A15D9B3796C
:104A300072791B021343F27912041A43337A1B066C
:104A400013433B603B68052231002000039306F0CE
:104A50007FFE0422601D03A96CE7FE236370F1E76B
:104A6000FC5BFF1FE8B80011305CFF1FFC0C00006E
:104A7000DCB80011F50C0000085CFF1FE85BFF1FAD
:104A8000B43DFF1F803CFF1F2C5CFF1F3C5CFF1FE1
:104A90006509FF1FADAC00002D5EFF1F2B5EFF1FE1
:104AA000AEDE000070470000020010B5094B0A326C
:104AB000094C92B2DA815A8298811882207802F0E9
:104AC00073F90422054B012120781A7006F0C0FC0E
:104AD00010BDC0463E3DFF1F765EFF1F755EFF1F87
:104AE000013870B5042809D806F0C2FC0309230870
:104AF00012001E4B0221187806F0AAFC70BD1B4B59
:104B00000821187806F04CFE0022194B1A72F5E7BE
:104B100080220024164B154D52001A810821287856
:104B20001A68DC7206F074FC2100287806F0E0FCBC
:104B3000E4E70E4B0821187806F032FE0D48FFF727
:104B4000B3F80D4B0D4A9B7993800D4A13800022D8
:104B5000074BDA720132FF321A810A4B5B78002B65
:104B6000CCD0094A136006F003FEC7E74C5CFF1F78
:104B7000205CFF1F893CFF1F305CFF1F3C3EFF1F76
:104B80007A3CFF1F2C5CFF1F34F0004010B5002959
:104B900004D1042802D10D3005F04AFA10BD0000FE
:104BA00010B501290ED104280CD10D3005F040FAC2
:104BB000054B1B78002B05D02622044B04485A7263
:104BC000FFF772FF10BDC0464E5EFF1F205CFF1F47
:104BD000C40900000300F0B50A4D8E18B14202D19D
:104BE00052008018F0BD0C782F6824093C5D0F2717
:104BF0001C700C7801313C402F683C5D5C700233C6
:104C0000ECE7C046743CFF1F0D22114B10B51A7023
:104C10000C23104C10492370093A033B0F48637072
:104C200006F096FD2D2301220D490E48A371FFF7D2
:104C3000D1FF01220C49FFF7CDFF01220B49FFF7FD
:104C4000C9FF00220A491000FEF7D6FA10BDC0467F
:104C50004A5EFF1F2B5EFF1F9BB800112D5EFF1FDA
:104C60006709FF1F325EFF1F6609FF1F6509FF1FEF
:104C7000AEDE000070B5124C132220001149FEF781
:104C800081FB114D002817DDAB78002B14D0431C9D
:104C90002B7009236B7000230019037028782900FA
:104CA0000130C0B206F0DCFB297822000139C9B21C
:104CB000002005F011FC70BDFFF7A6FFEEE7C0462F
:104CC0002D5EFF1FAEDE00002B5EFF1F10B5114BE7
:104CD0001A781870002A0ED000280BD10E4B1A78C3
:104CE000062A07D85423D340DB0703D50B4B18788B
:104CF00002F05AF810BD0028FCD0074B1B78012B9E
:104D000002D0033B022BF5D8044B0121187806F0A2
:104D10009FFBEFE74E5EFF1F755EFF1F765EFF1F76
:104D200070B54D4E4D4A4E493070042005F076FA6C
:104D30000021112005F07CF9112005F05DFAFEF745
:104D40005FF906F0EDFB032246494748FFF742FFB3
:104D50002D24030004221C7044490130FFF73AFF60
:104D600030230470424D434C437083702E3B062227
:104D700020004149EB87FEF705FB062813D02000F1
:104D800006F08EFA022809D00321200006F0A0FCCC
:104D90008D23E3706E3B237119336371062220006B
:104DA0003549FEF729FA354B1B68FC335C64FFF785
:104DB00061FF0020FFF78AFF314C324A0121324B5C
:104DC0001278207801F0B2FF304A314B127800217E
:104DD000207801F0ABFF01222E4B1A702E4B9B78EE
:104DE000552B31D12D4B3B325A722D4B2D4AAB8175
:104DF000EA812B826A822021307806F0A1FA012014
:104E0000404205F0B5FB0120404205F051FCFFF7A0
:104E10006BF9FEF72DFF00F09DFC01204042FEF7EC
:104E2000F5FF012006F07CFAF02001F03BF90121AA
:104E3000307806F00DFB307802F012F91A4806F0CF
:104E40005FFCFEF731FE70BD6422184B5B79534363
:104E50001A000A32CBE7C0464C5CFF1F8D4B001195
:104E6000A14B0011B43DFF1FE85BFF1F085CFF1F53
:104E70003E3DFF1F6509FF1FADAC0000985EFF1FA0
:104E8000765EFF1FA83CFF1F893CFF1F4A5EFF1F85
:104E90002B5EFF1F1C5EFF1F2C5CFF1F205CFF1F93
:104EA000C4090000CE0900004E5CFF1F305CFF1FEC
:104EB000F8B50A0020230D001A40194251D0534B77
:104EC0001B78002B3CD0FFF711FB514B514C524E3D
:104ED00099686268737A8A1ADB039A4202D3616026
:104EE000FEF7E2FD327A217A531EDBB299422AD1D3
:104EF000FFF7B2F9637A002B1FD0013BDBB263727C
:104F0000002B1AD1454B9B78552B01D106F030FC74
:104F1000E37A002B0CD00023414A424FE3721388FE
:104F2000380001331380FEF7BFFE390006F088F920
:104F3000642370795843FFF7B7FD237A0133237256
:104F400020206840F8BD9142D4D300232372FFF79C
:104F5000ADF9344F3800FEF7A7FE390006F070F9BE
:104F6000C8E70BB2002B0ADA2F4B187806F048FB83
:104F7000002801D006F0A4FB80200002E1E7022413
:104F8000214206D0234B01201A72FFF79FFE20001A
:104F9000D7E70B071BD5FFF7A9FA1D4B1D491E4C80
:104FA00098684A68637A821ADB039A4202D348609F
:104FB000FEF77AFDFFF77AF9FFF74EF900F0E4FB10
:104FC0002368DB0701D5FFF719F80820B9E710249B
:104FD000214206D00D4B1B78002BD8D1FEF75CFE8A
:104FE000D5E70124214209D0104800F06DF806F001
:104FF000E7FB2100112005F01BF8C8E70424080096
:10500000204021429ED0FEF71DFFC0E74E5EFF1FED
:105010003C5CFF1F205CFF1F305CFF1F2C5CFF1FF0
:10502000145CFF1F893CFF1F4C5CFF1F6C3CFF1F83
:10503000F0B51B4B1B4F1B883A8804001A4E1B4DC2
:1050400085B09A420DD832889A420AD3184B1A88F2
:105050002B889A4205D1174A174B12881B889A420F
:105060001BD0052001F074F83B8802AA1380338816
:10507000019053802B88114D93800F4B02A91B8800
:10508000D3800F4B2A78188802F090FD0D4B082131
:105090002878019A1C7006F0A3F805B0F0BDC04650
:1050A0001A5EFF1F7E3CFF1F7C3CFF1F7A3CFF1FE8
:1050B000185EFF1F165EFF1F783CFF1F765EFF1F06
:1050C000803CFF1F145EFF1F13B50C4B1C78002C97
:1050D00011D1002801D00A4B18600A4A0A4B1178F6
:1050E0000A4A10780A4A01920A4A0092002205F000
:1050F000EBF8200016BD1124FBE7C046755EFF1FCC
:10510000105EFF1F745EFF1F645EFF1F765EFF1F51
:10511000505EFF1F545EFF1F10B5064B12201B7818
:10512000052B06D1044B13221988044B187801F083
:10513000EBF910BD755EFF1F803CFF1F765EFF1F01
:1051400010B500240122114B52421870104B1C70F4
:10515000104B1A8001F084FF04220F4B21001A70BB
:105160000E480C3206F04CF8102221000C4806F0D4
:1051700047F807220B4B1C600B4B1C700B4B1C7031
:105180000B4B1A700B4B1C7010BDC046765EFF1F98
:10519000755EFF1F803CFF1F745EFF1F645EFF1F74
:1051A000545EFF1F505EFF1F2A5EFF1F295EFF1F18
:1051B000823CFF1F285EFF1FF8B5174C06002578BC
:1051C00006A814240078052D23D1B41F134FA5B2CF
:1051D0001824BD421DD88D1FADB2BD4219D8FA2585
:1051E0006D00AA4215D21D000D4F0A3DADB2BD4261
:1051F0000FD80C4C26800C4C21800C4900240A80CE
:105200000B4A1380FFF714FF0A4B0421187806F0AD
:10521000C7FA2000F8BDC046755EFF1F790C00007C
:10522000750C00007E3CFF1F7C3CFF1F7A3CFF1F7B
:10523000783CFF1F765EFF1FF0B50BB20D0089B002
:10524000002B00DB70E1A44E307806F0D9F9041E83
:1052500050D00378A22B00D122E1D02B1AD0912B71
:1052600045D143780E2B42D19C4B82889A423ED145
:105270009B4A83681278052A39D1032018567F2863
:1052800035D0984B1B68002B31D05B68002B2ED09B
:1052900098472CE08078072829D806F0E9F80428F8
:1052A000183F3F74A8D86378002B0CD101218C4B98
:1052B00019708D4B1A78002A5BD08C4B307801F036
:1052C00035FD002855D00722854B1A7051E06178D2
:1052D0000029F8D1E378002B11D0854A854B12784C
:1052E000307801F023FD60706378002BEBD1200053
:1052F00006F0E6F980200002684009B0F0BD784B66
:105300001B78022BF3D00121307806F041FA0028F7
:10531000EAD10121307806F09BF8E5E76378002BAD
:10532000D1D16F4F032807D13B78052B02D1013330
:105330003B701EE00223FBE76F4B1A886F4B029312
:10534000002A0BD01B78002B03D00121307805F008
:1053500047FF3B78062B04D1013BE9E7029B1A701B
:10536000F7E7042B41D10121029B3078197006F038
:105370006FF85C4B1B68002BB9D01B68002BB6D0B4
:10538000574A107884E76378554F002B27D10622BF
:10539000211D5B4806F0DCF962895A4B5A491A8094
:1053A000A2895A4B1A80E3890B800521397058492C
:1053B0000A80584A1380228A574B1A80574B1B7811
:1053C000012B09D11F2000F0C3FEFA2292004243B4
:1053D0000421307805F004FF0022484B75E7312B9B
:1053E00000D070E70022454B1A700323A0E7062285
:1053F0000021434805F004FF0023454A042113809F
:10540000444A30781380444A138006F0C9F90821D1
:10541000307806F0C5F9A379083B5A425341304A27
:1054200003331370304B1B78002B06D0334B30788E
:105430001A78002A06D001F0B7FC0122314B524203
:105440001A8096E70121197006F002F8F5E70821A5
:10545000307806F0A5F96378002B00D047E72C4B95
:105460002D4F0293E388029A04211380294B307850
:1054700003932389039A138063893B8006F088F99C
:10548000002800D033E7264B1B68002B00D12EE705
:10549000039902983A88098800881B68984726E78C
:1054A0004379132B00D022E70389012B0AD11D4B2E
:1054B0001B78022B06D10821307806F071F9FFF72E
:1054C0002BFE14E7052000F043FE0821020030788F
:1054D00005F086FE0BE7C046765EFF1F0514000050
:1054E000755EFF1F105EFF1FA83CFF1F893CFF1F5A
:1054F0004A5EFF1F2B5EFF1F4C5EFF1F4E5EFF1FAD
:105500001D5EFF1F803CFF1F245EFF1F265EFF1FE6
:105510001A5EFF1F185EFF1F165EFF1F1C5EFF1F37
:105520000C5EFF1F145EFF1F8020C001014200D0EF
:10553000E2E6CB0731D5324B1B78002B1DD0314E24
:1055400005AC3378052B1AD1023B23702E4B21007A
:105550001B7823722D4B1B7863722D4B187801F04A
:1055600089FB002809D007202A4B30701B68002BCC
:1055700003D01B68002B00D098470120BCE60E200A
:10558000254B06221B7825492370254B1B78637019
:1055900002ABC01806F0DCF8D8E702230800184078
:1055A000194209D0174B1B78052B03D11D4B1888C6
:1055B00005F02EFE02209FE60424214203D0FFF7CF
:1055C00037FD200098E6082308001840194200D152
:1055D00093E6154B1C78012C03D0022C0DD008202B
:1055E0008AE6124B124A134913481B88128809880D
:1055F00000880094FFF7E0FDF1E7FFF78DFDEEE78F
:105600004E5EFF1F755EFF1F823CFF1F285EFF1F5F
:10561000765EFF1F105EFF1F2A5EFF1F833CFF1F89
:10562000295EFF1F803CFF1F145EFF1F783CFF1F99
:105630007A3CFF1F7C3CFF1F7E3CFF1F10B502A879
:1056400004880B20002C10D1496808784978090299
:1056500001430C48814209D1022119800A4B598823
:105660001170DB7800205BB2537010BD074C0A202C
:10567000A142FAD102211980034B998811705B79FC
:10568000F0E7C0466E2A0000145CFF1F6F2A00007E
:10569000F7B5150008AA16884A680F4F1478527893
:1056A000120222430A24BA4214D10122DBB201922F
:1056B00000962A0005F00EFD041E0BD1074B1B6857
:1056C000002B07D068782A780002104342425041EC
:1056D000013098472000FEBD02290000885EFF1FB0
:1056E00030B5012503790400BFB02B4225D0144901
:1056F000408805F05BF828420CD0124B01A95B8D65
:1057000000220B8002234B800F4B5B888B806088CC
:1057100002F042F90D49608805F048F8C0070CD541
:105720000B4B01A91B8800220B8002234B80064BE8
:105730009B888B80608802F02FF93FB030BDC04657
:10574000805EFF1FAC3CFF1F145CFF1F785EFF1FD5
:10575000063DFF1F10B5074C0749200004F0DCFF91
:105760002000064904F0D8FF0721054A054804F047
:1057700095FF10BDFFFF0000805EFF1F785EFF1FDA
:1057800008B90011AC3CFF1F10B5024802F086FFBB
:1057900010BDC046E15600110200F0B501270A48CD
:1057A0000A4E51188B1A002B00DCF0BD0824157826
:1057B0004308684038404000805B013C58406D0819
:1057C000002CF5D10132EDE7FFFF000022B90011F6
:1057D000F0B500250F269D4200DBF0BD4C5D0709AA
:1057E00044403440A400A05801357840F3E700005D
:1057F000F0B589B06A460D000B000F271100103577
:105800001C780133260024093E4016705470023281
:10581000AB42F5D12023024AFFF7DAFF09B0F0BD11
:1058200028B90011F0B54E780B7889B036020C001B
:10583000170001901E43012A61D9954B9E4200D862
:1058400077E001339E421CD1062A17D1CA788B78A3
:1058500012021A430B791B0413434A7912061A43A6
:105860008C4B5A6100221A705A808B4A5A608B4ABC
:105870009A608B4ADA60002009B0F0BD8822520598
:10588000EEE7884B9E423CD182498B78002B00D0BA
:10589000F6E00C2A31D10F22A3789343E27812026A
:1058A00013432279120413436279120613434B60A7
:1058B000E279A07912020243207A00041043627A4E
:1058C00012060243CA60E27AA07A120202437648C4
:1058D0004A81834208D804236E49142201980B7030
:1058E00005F036FF1420C7E71201D21889235B05A3
:1058F0009A42F0D801238B70BDE7022AFAD0052323
:10590000EAE76A4A01239642E6D1FFF705FC052F34
:105910000CD9E378A2781B021343227912041A43AC
:1059200063791B061343624A0393136005F020FF5B
:10593000A1E7584D2B78002B9DD1AB78002B00D1DF
:10594000A0E02B8901339BB20093B34200D091E0D9
:10595000132AD4D9CF7C8B7C3F02122120001F4315
:10596000FFF71AFF874200D08EE0002E3DD1E3788A
:10597000A2781B0213432279E96812041A4363795F
:105980001B06134303930A228B4212D1FF23A370F9
:10599000E370237163716B89002B09D1E37B227C57
:1059A0001B0212041343A27B13431B0901336B81B7
:1059B00000226B89002B8ED0002A67D168683701DE
:1059C0003818000B6B6900030390984205D9686191
:1059D00005F0F6FCEB780133EB7068681022A11C2F
:1059E000381805F01DFD2E8145E76F89009A7B1E52
:1059F0009BB293423AD1E278A37812021A432379F8
:105A000005A81B04134362796C6812061A43EB68FD
:105A100000920392211D0C22049305F099FE0120AF
:105A2000260004A940421036FFF7E2FE013F012F95
:105A300017D1009A0B232861824200D04CE7042240
:105A40001C49200005F0ECFC042203A9686805F05D
:105A5000A7FBE968039AFF23914200D13CE7F73B9B
:105A60003AE73100FFF7C4FE1036DFE70923B742FB
:105A7000A4D831E7009BB34200D9FCE607232BE70B
:105A8000022329E7032327E7062325E70A2323E741
:105A9000FFFE0000203DFF1F00000111FFFF00007E
:105AA0005048593601FF0000FFFF001102FF0000BF
:105AB00034F000402C3DFF1F10B5034C0B000122B9
:105AC000210000F06BFA10BD795C00110B8870B5F5
:105AD00006000D000224162B11D92B0003220949C0
:105AE00000F05CFA041E0AD1074B2A881B88191C97
:105AF000934200D9111C300089B200F0EFFA200067
:105B000070BDC046A55C0011B25EFF1F10B54A789B
:105B10000400013A0B000220012A07D80A78002A63
:105B200004D005222000024900F038FA10BDC0461A
:105B3000D35C00110A7810B50B0004000220002A83
:105B400004D007222000024900F028FA10BDC04608
:105B50007F5D00110A7810B50B0004000220002AB6
:105B600004D009222000024900F018FA10BDC046F6
:105B7000E55D001110B5034C0B000B22210000F075
:105B80000DFA10BD155E001110B5034C0B000D226F
:105B9000210000F003FA10BD875E001110B5034C20
:105BA0000B000F22210000F0F9F910BDE15E001199
:105BB0000A7810B50B0004000220002A04D011223C
:105BC0002000024900F0EAF910BDC046F15E001164
:105BD000002310B51322190000F0E0F910BD0000F9
:105BE00010B5034C0B001722210000F0D7F910BDAF
:105BF000435F0011002310B51922190000F0CEF9FF
:105C000010BD000010B5034C0B001B22210000F05A
:105C1000C5F910BD7D5F0011F7B584890D00060040
:105C20000121002C22D000238268D3561778002B44
:105C30001EDA0C2C1AD90C3CA4B21319408800931C
:105C4000230002F086FE431E984101307B06DB0FE5
:105C50006B703F23013C1F40A4B22870AF70AC8032
:105C6000002C07D0B3680133AB6000210800FEBDF3
:105C70000020EBE7AC60F8E70B7803704B884370CB
:105C80004B881B0A83700B79C37004207047042073
:105C9000022B06D10020537811781B02009A0B4387
:105CA000138070470B8803700B881B0A4370022017
:105CB00070470420009983420AD1537810781B0260
:105CC00003430B80D37890781B02034300204B8062
:105CD0007047F8B50D004B7801240021461C037075
:105CE0002B788B4201D82000F8BD6B78B01C4F1C7C
:105CF000012B10D1890069184B88022233704B8820
:105D0000B9001B0A7370691805F062FA043604348E
:105D1000A4B2F9B2E4E7122359436B185A8804314C
:105D200032705B8810221B0A7370691805F050FAF4
:105D300012361234ECE770B5049D14001E00052BDA
:105D400001D8042070BD637812781B0213432B80A6
:105D5000E378A2781B02134302226B802A71211D73
:105D6000681D063E05F034FAB2B22A81E92AE8D865
:105D70002800A11D0A3005F02BFA0020E2E70023DD
:105D800010B50A789A4201D8900010BD9A008A187E
:105D90005488013304705488DBB2240A4470948818
:105DA00084709288120AC2700430EAE710B51100BC
:105DB000029C062B04D004201022142B01D010BD0D
:105DC000022222714B7808781B0203432380CB7890
:105DD00088781B02034363800431601D05F0F8F9E5
:105DE0000020ECE710B50C788B7804315C43E4B20A
:105DF00003702200013005F0EBF9601C10BD042097
:105E0000022B06D10020537811781B02009A0B4315
:105E10001380704710B50C000A88023105F0D8F9DC
:105E2000208810BD70B504000D0004981100012BEE
:105E300001D8042070BD16785278120232430280D5
:105E40000200F13255701470E125002C00D10C35A0
:105E5000023B9AB24280AA42EBD80231043005F0EC
:105E6000B7F90020E6E70420009983420AD153786D
:105E700010781B0203430B80D37890781B020343F6
:105E800000204B80704710B50C000A88023105F0E5
:105E90009FF9208810BD000070B501211E0004206C
:105EA000049C0E400B4218D1CB40DDB28D4214D978
:105EB0000A49DBB2098899420FD32300EE331D70E3
:105EC0003300580011184978165C09023143013338
:105ED0002152D9B28D42F4D8002070BD383DFF1F49
:105EE00010B50C000A88023105F072F9208810BD47
:105EF00010B50C788B7804315C43E4B20370220057
:105F0000013005F065F9601C10BD10B51100029854
:105F1000032B01D8042010BD14785278043B1202E0
:105F200022430280CA788C781202224342809AB2BD
:105F30008280EB2AEED80431063005F049F90020C2
:105F4000E9E710B50C000B8803700B881B0A43703F
:105F50004B8883704B881B0AC3708A8804300631D3
:105F600005F036F9A088043080B210BD0420012B62
:105F700003D100201378009A1370704710B50C00FD
:105F80000B8803700B881B0A43704A880230043167
:105F900005F01EF96088023080B210BDF0B589B0FE
:105FA00003931E4B029242000700D05A019102F067
:105FB00020F81325061E2DD0029B01240370019B9F
:105FC000002B04D0001903999847001984B26B463E
:105FD0001B7A5BB2002B0FDA1021380002F01CFB99
:105FE0001925002813D130003219E1B202F066FC05
:105FF000051E0CD10C34A4B2042304AA380005A950
:1060000093800696948101F0AFFD051E02D030000A
:1060100005F076FA280009B0F0BDC046B05EFF1F5B
:1060200070B505000C0000280CD00020814209D07A
:1060300010222000044905F0CBF801202B782373AF
:106040006B78637370BDC04668B90011F0B5060087
:106050000D0017001C0085B002291BD0002010295C
:1060600007D1022B07D0102B03D115E00020102CF4
:1060700008D005B0F0BD69463800FFF7D1FF2A000F
:1060800069460BE069463000FFF7CAFF2200694607
:10609000380004E0022BE9D12A003900300005F075
:1060A000EFF9E6E7031CF02800D9F02303200849A4
:1060B0009AB2013A0B80D317034006499B189B10F4
:1060C0000B80D30F04499B185B100B807047C046B0
:1060D0003C3DFF1F3A3DFF1F383DFF1F034B1B8810
:1060E0008B4202D3024B4000C15270473C3DFF1F20
:1060F000B05EFF1F014B4000185A7047B05EFF1F93
:106100001722014B1A807047B05EFF1F70B5050063
:106110000E2005F0BDFA041E13D0D0230370002317
:106120000622837007494570033005F051F8064B8D
:106130002100DA8A62811B7E2373044B187805F0F4
:106140001FF970BDCC5EFF1FBC5EFF1F8C3DFF1FA3
:10615000262803D8024B4000C05A70470148FCE78C
:106160003E3DFF1FFFFF000070B506000C00094D0B
:106170001C220021280005F043F8074B1E70074B36
:106180001C7005F0D5F90123002801D0002312204E
:106190002B7070BDBC5EFF1F8C3DFF1FDD5EFF1FBF
:1061A00070B505000D4C0800E260A16010220021CE
:1061B000656005F065F8012803D11021A06802F0A0
:1061C00058FD10220021280005F05AF8012803D1BB
:1061D0001021606802F04DFD70BDC046BC5EFF1F1F
:1061E00070B5041E05D1002903D006220D4804F025
:1061F000EFFF0D4B1D78012D11D1002C05D102228E
:106200001A7005F025FA280070BD00221A70074B9D
:106210001B78FF2BF7D02000FFF778FFF3E700256E
:10622000F1E7C046CC5EFF1FBC5EFF1F8C3DFF1F29
:10623000030010B5002801D1002010BD00780B4AE2
:10624000002803D15988D1821B7913761378022B49
:10625000F2D10023984200D103331370044B1B7812
:10626000FF2B01D0FFF752FF0120E6E7BC5EFF1FC6
:106270008C3DFF1F002911D000280CD04B7901283C
:1062800003D140225242134303E03F22134003282C
:1062900002D001204B7170474022F4E70800FAE772
:1062A00070B5094D0100287800280BD0074C062254
:1062B000200004F08DFF21002878FFF7DBFF20008D
:1062C00005F00EF970BDC046DC5EFF1FB65EFF1F15
:1062D00000290AD0012808D13F224B799343C02BD3
:1062E00003D0403B5A425341981C704770B5174D3C
:1062F00006002B78FF2B15D00A2005F0C9F9041EE3
:1063000010D0D0230370C83B8370114B11491B7808
:106310004670C3700622043004F05AFF210028782A
:1063200005F02EF80C4B1B78012B0DD10B4B1B6885
:10633000002B03D09B68002B00D09847084B04210A
:106340001878084A05F064F870BDC0468C3DFF1F00
:10635000DC5EFF1FB65EFF1FD85EFF1F045FFF1FDE
:10636000085FFF1F60EA0000014B98687047C04655
:10637000BC5EFF1F014BDB6818687047BC5EFF1FE7
:10638000074B10B5DA68136801331360054B1878B2
:10639000FF2803D08021C90105F05AF810BDC0467E
:1063A000BC5EFF1F8C3DFF1FF7B50E0002F0C8F862
:1063B000051E1CD00E4B06621F78002F00D10778F7
:1063C000AB791020019305F063F9041E0FD0D023A0
:1063D0000380C73B8370019BE91DC3700622043014
:1063E00004F0F6FE21003800E66004F0C9FFF7BDB6
:1063F0008A3DFF1F014B18787047C046DC5EFF1FC7
:10640000054B002805D1054B1A78054B002A00D111
:10641000014B18007047C046CC5EFF1FDC5EFF1FBB
:10642000B65EFF1F014B58687047C046BC5EFF1F39
:10643000024B1868431E9841C0B27047E05EFF1FD0
:10644000421E03000120152A03D9FF3B5A42534143
:10645000D8B27047F0B51C0000230E0085B0039041
:1064600002920B70029A934201D3002019E0E55C7E
:106470005A1CD2B2002DF8D0029851198142F4DC96
:106480000233DFB2A35C18000193FFF7D9FF0028A5
:1064900007D0013D019A0399EBB233708A4202D1D1
:1064A000E01905B0F0BDDB19DBB2DBE710B50C007D
:1064B00002F09EF803001220002B03D02100588820
:1064C00004F006FF10BD000070B50E4D8400635946
:1064D000002B15D0186A002801D005F0D1F82B59EF
:1064E000586A002801D005F0CBF82B59986A00288B
:1064F00001D005F0C5F8285905F0C2F800232B514A
:1065000070BDC046EC5EFF1F1C4B70B504000E0052
:10651000150099420AD11A4B1B68002B01D1122099
:1065200070BD1B68002BFAD09847F9E7154B9942CC
:1065300015D1134B1B68002B0AD01B68002B07D00A
:106540009847002804D1104B1C70104B1D70E7E7D2
:1065500029002000FFF7AAFF0028E1D1F3E7080097
:1065600001F0EEFF0028DAD003780320A342D7D150
:106570002900300004F0ACFED2E7C046FEFF000068
:10658000E85EFF1FFFFF0000E55EFF1FE45EFF1FE8
:10659000F7B50400808801F0D3FF0025A84203D09E
:1065A0000578A08802F008F81C4E3378002B1FD025
:1065B000AB421DD11A4B28001978FFF777FF00284E
:1065C00018D000233370A3790820A778A6880193F8
:1065D00005F05EF8011E0DD0D0230370CA3B837016
:1065E000019B477086808371280004F0C9FE01E09A
:1065F000002DE8D1A0880B4B8200D358002B01D08E
:10660000FFF762FF1721A088FFF768FDA08801F05F
:1066100027FDA08801F0FEFDF7BDC046E55EFF1F27
:10662000E45EFF1FEC5EFF1FF0B587B01D000CABF2
:106630001B88070001930DAB1B88142002930EAB3F
:106640001B88160003930FAB1B880091049310ABBB
:106650001B88059305F01CF8041E1AD0D023037084
:10666000CB3B47708370C670062229000430002D92
:1066700011D004F0ADFD019B21006381029B0098C5
:10668000A381039BE381049B2382059BA37404F0F5
:1066900077FE07B0F0BD04F0B3FDECE7F7B500936B
:1066A00008AB1B8807000C200D001600019304F0B6
:1066B000EFFF041E13D0280001F042FF00280FD086
:1066C0000078D0232370C93BA370009B2100238155
:1066D000019B6770A580E680638104F051FEF7BDE1
:1066E000014B1878EDE7C0468C3DFF1F13B5040041
:1066F00064890389C2888188C0780094FFF7CEFF3F
:1067000013BD000010B5044C2068002803D004F02D
:10671000B7FF0023236010BDF05EFF1FA122F0B57C
:10672000818892004A43384B384F1B6804009B18FD
:106730009D2292009B18827989B01A603B68002BD9
:106740005FD01D78324B1B68002B04D05B68002B98
:1067500001D000209847260008363100E079FFF785
:10676000B7FD237DE0710200E0780493638A29007D
:106770000393238A0293E3890193A3880093330050
:10678000FFF752FFE378002B0BD1E289A379A188B0
:1067900002920196E27928000092012201F0DAFECD
:1067A000E0703B68002B20D0FFF7ACFF194D287834
:1067B00000281AD0184B1978FFF778FE002814D05B
:1067C0002B78E67808200793A78804F061FF011E64
:1067D00009D0D0230370CA3B4670837087808671CE
:1067E000079804F0CDFD00232B701721A088FFF738
:1067F00075FCA08801F034FCA08801F00BFD09B005
:10680000F0BD064B9DE7C0463409FF1FF05EFF1F39
:10681000045FFF1FE55EFF1FE45EFF1F8C3DFF1F4F
:10682000F8B5070008000E0001F08AFE041E18D01B
:106830002620FFF78DFC051E00D12578062004F0E8
:1068400027FF041E0DD00021062204F0D9FCD0231E
:106850002370C23B21006770A370A680E8B204F0E9
:106860008FFDF8BDF0B585B001930AAB1B7807002A
:1068700002930BAB1B7808000D000092039301F00C
:106880005FFE061E22D0102004F002FF041E1DD061
:106890001022002104F0B4FC2620FFF759FC002848
:1068A00000D13078D0232370C13BA370009B21001E
:1068B0002372019B67706372029BA580A372039B86
:1068C000C0B2E3720C9BE36004F05AFD05B0F0BD6A
:1068D000F7B50D00019001F033FE071E20D00E2009
:1068E00004F0D6FE041E1BD02620FFF731FC061E46
:1068F00000D13E78D0232380C53B0622A370F91D2A
:10690000E01C04F065FC019B2A0063810123DD404B
:106910001A401D40210022736573F0B204F030FD6F
:10692000F7BD0000F0B585B0029010000D00170013
:106930000A9E039301F004FE041E31D0029B002B3B
:106940002ED1039B02795B0724D512231343042223
:10695000002E08D10B99002905D10C99002902D1EC
:106960000D9900291AD01A430D9B2271002B00D0DB
:10697000C9E0002E00D1CFE0002D00D0CCE0606A4D
:10698000002801D004F07CFE1C21300004F030FD12
:10699000606205E002239A430E33D7E793432371E5
:1069A000654BBA00D458002C00D1AAE0002E10D0BC
:1069B000236A002B03D11C2004F032FE20625E4BC0
:1069C000BA00D358186A002803D01C22310004F002
:1069D000FFFB0C9B002B12D0574CBB001D596B6A60
:1069E000002B03D1162004F01BFE6862BB00E358A5
:1069F000586A002803D016220C9904F0E9FB0D9B7D
:106A0000002B11D04C4DBC006659B36A002B03D14A
:106A1000142004F005FEB0622B59986A002803D0B8
:106A200014220D9904F0D4FB380001F089FD051EF5
:106A300067D0414BBA00D358002B62D01A6A342079
:106A4000002A00D11C389A6A002A01D0143080B282
:106A50000B9A002A01D01C3080B25B6A002B01D057
:106A6000163080B204F014FE041E4AD01822002111
:106A700004F0C6FB2620FFF76BFB0190002801D134
:106A80002B780193D0232370029B200063700A238C
:106A9000294EA370039BBD00A371AB59A780196A4F
:106AA0001830002905D01C22A06004F091FB2000C2
:106AB00034307359996A002907D003001422143323
:106AC000E060029304F084FB02980B9B002B08D03B
:106AD00003001C221C330B992061029304F078FB05
:106AE00002987359596A002903D01622606104F094
:106AF0006FFB6B462100187904F042FC3800FFF769
:106B0000E3FC05B0F0BD10220D9B0D991B69A01888
:106B1000236204F05DFB2CE70B9B002B00D13FE7C9
:106B2000012D00D03CE7606A002801D004F0A8FDE8
:106B30001C210B982AE7C046EC5EFF1F10B5044CE1
:106B40002068002803D004F09BFD0023236010BDC3
:106B5000E05EFF1F0B4B07B51A68002A01D1002029
:106B60000EBD6946531C012012780731FFF772FCF5
:106B70000028F4D002780123100018401A42EED009
:106B8000EEE7C046FC5EFF1FF0B51F4F01203B68DB
:106B900087B0002B25D09B78059300F0B3FB00282D
:106BA00021D00A20FFF7D4FA04000B20FFF7D0FA17
:106BB000164B05001E78731E9E413B68F6B2191DE8
:106BC000D878FFF757FB3B682900DA7A0433039241
:106BD0009A7901930292009033002000059A04F004
:106BE0005FFD07B0F0BDFFF7B5FF002805D0062018
:106BF000FFF7AEFA04000720D8E70820FFF7A8FA4D
:106C000004000920D2E7C046E05EFF1FDC5EFF1FE4
:106C100070B50A4E040033780D00FF2B0DD0042010
:106C200004F036FD011E08D0D0230370CE3B457022
:106C30008370C470307804F0A3FB70BD9C3DFF1FCF
:106C400070B5040006200D0004F022FD011E0AD0DC
:106C5000D0230370CD3B8370054B44701B68858047
:106C6000187804F08DFB002C01D0FFF767FF70BD92
:106C7000E05EFF1FF8B5264F06003B680D001124AB
:106C8000002B05D10522234B1B78134202D112247D
:106C90002000F8BD204A10241268002AF8D012788B
:106CA000002AF5D0DB0719D52B789A1E012A1AD8AD
:106CB0000C2004F0B5FC132438600028E8D0002331
:106CC0000A22437029000670023004F081FAFFF7AF
:106CD0005BFF041E0AD0FFF731FFD9E700F012FB7B
:106CE0000028E1D1E4E7002BE2D0D0E70B4B1B7882
:106CF000032BCDD11D20FFF72BFA094B188000285C
:106D0000C6D0084B04211878074A04F081FBBFE77E
:106D1000E05EFF1FDD5EFF1FFC5EFF1FDC5EFF1FEE
:106D2000DA5EFF1F085FFF1F60EA0000F7B50193FE
:106D3000194B14001A78052306000F0012201A427E
:106D400021D0012920D1154B1D68002D1BD0022018
:106D50001F2C18D8002C02D0019B002B13D0104BF5
:106D60001F221E706E1C0021300004F049FA0199A8
:106D70002200300004F02CFA310020002C70002F8B
:106D800006D004F0ADFAFEBD064B12201D68DCE70C
:106D900004F066FBF7E7C046DD5EFF1FFC5EFF1FE9
:106DA0009C3DFF1FF85EFF1FF8B50F4E122433689D
:106DB000002B17D01B780F3C834213D100250B4FBB
:106DC0000221387804F0ECFC094B042138781D804E
:106DD00004F0E6FC074B28001D8033685C7004F06B
:106DE000A7FA04002000F8BDE05EFF1F085FFF1F48
:106DF000F45EFF1FDA5EFF1F70B5012823D11B4C24
:106E00002388002B03D01A4A1578002D07D0194B80
:106E10001B68002B02D01878FFF7C6FF70BD3B2B14
:106E200002D93C3B2380F9E7134E0221307804F06D
:106E3000B7FCFA222388920002215A43307804F0EA
:106E4000CFF92580EAE70B4B1B68002BE6D00B4BF4
:106E50001B785B07E2D5084B0221187804F0A0FCF0
:106E60000022024B1A80FFF769FED7E7F45EFF1F8E
:106E7000D85EFF1FE05EFF1F085FFF1FDD5EFF1F84
:106E8000F8B51E4D2868002803D004F0F9FB002354
:106E90002B601B4E3068002803D004F0F1FB002368
:106EA0003360184F05243B7818002040234221D03E
:106EB000154800F02BFA3B78234213D0202004F031
:106EC000AFFB2860002813D02022002104F098F99D
:106ED000202004F0A5FB041E306005D020220021F4
:106EE00004F08EF9002004E0286804F0C9FB2C604F
:106EF0001320F8BD00F00AFAF4E7C046FC5EFF1F5D
:106F0000F85EFF1FDD5EFF1F903DFF1F10B50A4CAE
:106F100023681A1E0ED0002808D10130587004F0E2
:106F200007FA002805D02368002B02D00021FFF7C4
:106F300087FE0122100010BDE05EFF1FF7B5274E4F
:106F4000050033680191181E21D05C78244F012C74
:106F500030D1FFF7FFFD002825D02000FFF7F8F81B
:106F60000400412814D91F4B022118781E4A04F04E
:106F70004FFA1E4B3C3C1C80022233685A703B780F
:106F8000002B14D128000199FFF75AFE0120FEBD05
:106F9000FA2292004243002AEED0124B02211878C6
:106FA00004F01EF9E8E7FFF7D3F80200F3E7002347
:106FB0003B70EBE73B78002BE8D1032004F068FB43
:106FC000011E08D0D0230370CC3B4570837033681A
:106FD000187804F0D5F9FFF7B1FDD7E7E05EFF1FA1
:106FE000D85EFF1F085FFF1F60EA0000F45EFF1F0E
:106FF00010B51749838802008B4220D011D815495B
:107000008B4217D0144900205B1899B2012907D888
:10701000926811785A425341D8B2FFF7F9FD012026
:1070200010BD0E4A00209B1807229BB29A42404195
:10703000C0B2F5E783681878FFF768FFF0E7836868
:1070400099785A78090218781143FFF777FFE7E734
:107050000A20000006200000F8DFFFFFAFDFFFFF7F
:10706000014B18707047C0469D3DFF1F10B5064C80
:10707000207001F041FA207804F092F9052120787F
:1070800000F062FD10BDC046085FFF1F0BB273B574
:107090000D00002B00DBC4E0884B187804F0B0FA38
:1070A000041E0ED00378912B0FD0A22B00D1A1E0AB
:1070B000834B1878FF2852D0210004F061F9002892
:1070C0004DD180200002684076BD43780F2B76D0EA
:1070D00013D8052B70D00E2BEAD18088794B9842BB
:1070E0002BD8794B98421BD8784B9842E0D1A368B3
:1070F0001878591CFFF774F838E03E2BD8D1837804
:10710000032B74D06CD8012B6ED0022BD0D1704BD6
:107110001B68002B23D05B68002B20D098471EE013
:107120006C4BC0180C28C3D804F042FB1DC2C2151A
:107130000BC20B0B0B3223C23C00674BC018072855
:10714000B6D8664B1B68002B09D01B68002B06D0F5
:10715000200098470AE0A3681878FFF7C7F82000D6
:1071600004F0AEFAADE7A068FFF762F800289FD000
:10717000F5E7A3681B78002BF1D0554B1B68002B5B
:10718000EDD01B68002BEAD0210055489847EDE769
:107190004F4B1B68002BE2D01B68002BDFD0210077
:1071A0005048F3E7504B1B68002BD8D05B68002B8E
:1071B000D5D021004348E9E7FFF7EAF9CFE7808817
:1071C0004A4B984203D04A4B984200D070E7464B56
:1071D0001B68002BC3D05B68002BC0D02100D5E713
:1071E000153B012BBBD963E7FFF798FAB7E7FFF729
:1071F0007DFAB4E73F4B1B78042B07D100236A4686
:1072000013800179408800F0C5FCA8E7364B1B6865
:10721000002BA4D05B68002BA1D001003648984712
:107220009DE7012421420AD0294B1B68002B04D082
:107230005B68002B01D000209847012043E78B07B3
:107240000AD5264B1B68002B04D05B68002B01D0AD
:1072500020009847022036E70421280008400D420C
:1072600000D131E7254E3388002B21D0013B9BB262
:107270003380002B1AD1FFF7DBF800280AD0204B0F
:107280001C70164B1B68002B04D05B68002B01D0D0
:1072900020009847FFF7C6F8694601F001FD6846EF
:1072A000FEF7FEFF1D20FEF753FF308004200AE7A3
:1072B000024B187804F074FAF8E7C046085FFF1F25
:1072C0009D3DFF1F0E20000001200000091000005E
:1072D000005FFF1FFEDFFFFFAFDFFFFF045FFF1F49
:1072E0000C2000000B200000E85EFF1F0D200000B6
:1072F00013200000DD5EFF1FFFFF0000DA5EFF1FAE
:10730000D85EFF1F10B501F09BF910BD014B18604E
:107310007047C046045FFF1F0B880020162B01D862
:1073200017230420014A13807047C046B25EFF1F36
:1073300000207047074A03001188814207D09188D6
:107340000020994202D101308000101870470020BF
:10735000FAE7C046105FFF1FF0B58F7806000D00FA
:10736000C5B01E2F15D1FFF7E5FF051E03D1002480
:10737000200045B0F0BD00223B003100C0780092F3
:1073800000F0B2FB0400A81C00F0D2FBFF23EB705E
:10739000EEE7264B062403931B78FF2BE8D0182F2B
:1073A000E6D87B08224A013BDB0002929A589446B9
:1073B000002ADDD0029AD3185B68002BD8D0087859
:1073C000002802D14B78012B02D10624122FCFD1F5
:1073D00007AFAB88697800976446AA68A047041E87
:1073E000C6D1AB78029A5B08013BDB00D3183900A9
:1073F00030005B689847041E0BD1AB78042BB6D0E5
:10740000039A310010782200009700F06DFB040011
:10741000AEE76A78002AABD1AA7805A93B88087143
:1074200030000A704B80FEF747FBA0E7A03DFF1F2E
:1074300078B900111D4B37B5050098420BD00029D3
:107440000AD1FFF777FF002805D11948FFF772FF2F
:10745000002800D0058037BD01291AD1FFF76AFF47
:10746000041EF8D001235B420380A378FF2BF2D0E7
:10747000FE2B07D00023E0781422009329001E334E
:1074800000F032FBA01C00F053FB01235B42638041
:10749000E1E70229DFD1013901F0BEF80028DAD195
:1074A0002800FFF747FF041EDFD1D4E7FEFF0000EE
:1074B000FFFF0000022210B5074B52421A80074816
:1074C00001325A809A80DA8000F07EFA044801F096
:1074D00025F8002010BDC046105FFF1F5973001132
:1074E000357400110388F7B50400002B02D1022582
:1074F0002800FEBD42680221137825485268FEF735
:10750000A5FD00282ED0234F01253A88002AEFD070
:10751000802321885B0201259B1A9942E8DC0C201C
:1075200004F07EF8061E31D03B8822889C4600235A
:107530001800019561469DB2491989B2AA421BD82B
:10754000002801D062443A8000233000082208C09D
:10755000210003F03DFE104A1368002B13D10025D3
:107560001660C5E76268022113780C485268FEF77E
:107570006DFD0028C7D1BAE760681D01401941813F
:1075800001330198D6E71A001B68E6E71325AFE739
:10759000E6B900119E3DFF1F0C5FFF1FE4B900110B
:1075A000014B18707047C046A03DFF1F14230A000E
:1075B00010B51A40194204D00122102101F048F8F8
:1075C00010BD4B06F9D4012088434000F8E710B500
:1075D00014008B0604D50122102101F039F810BDEA
:1075E00008230A001A40194202D14BB2002B0FDACD
:1075F000102101F02DF8002808D02300F2331B7869
:10760000002BECD0F1342378012BE8D10020E6E701
:1076100003208907FAD4E2E7F0B51F00184B85B0C4
:107620001C68019002910392002C27D1200005B024
:10763000F0BDA5683301ED186B89019A934211D30F
:10764000029A93420ED8002F04D10A9B002B10D12E
:107650002C00EBE73B002978039A6868FEF7F6FCFC
:107660000028F2D10136B6B2A388B342E1D824682B
:10767000DAE7A3680A9A5B891380E9E70026F3E753
:107680000C5FFF1F37B50C000A884988012391421F
:1076900017D3002A15D0651D23792A0002210A4834
:1076A000FEF7D4FC102300280BD0237961882088B2
:1076B00000242A000094FFF7AFFF0A23A04200D065
:1076C000230018003EBDC046E6B9001113B50A00FC
:1076D00008884988012388420BD8002809D0002453
:1076E000137905320094FFF797FF0A23A04200D0D8
:1076F0002300180016BD13B50A0008884988012325
:1077000088420BD8002809D0002413790532009450
:10771000FFF782FF0A23A04200D02300180016BD05
:10772000F0B58BB003904A8808880E00012382428E
:1077300055D3002853D00023012704AC2370002226
:10774000718813000092FFF767FF051E3ED0207876
:10775000002835D12B78022B18D167706A898300F5
:107760000130E31880005A8069680222201803F073
:107770002FFD23780133DBB22370042B19D93B0092
:107780006889013080B2002BD9D01FE002236370DA
:10779000122358436A89231804305A8069681022DA
:1077A000201803F015FD23780133DBB22370002B82
:1077B000E5D10C4A6B899B185A425341DBB2DFE793
:1077C0006378012BE4D12B78022BC7D022780A23CF
:1077D000002A04D021000398FEF798F9002318002E
:1077E0000BB0F0BD0100FFFF0F4BF0B504001868AF
:1077F000002816D083685D89A54207D88288AE1814
:10780000B44203DA12019A18934201D10068EFE7FB
:107810001E005F891036A74204D1002900D00D80D8
:107820001800F0BD3300EFE70C5FFF1F70B50500D7
:107830000C0008880021FFF7D7FF03000120002B70
:1078400004D022002800197AFFF7C1FE70BDF7B5F9
:107850000C00002501902300EE331B78AB4201D8C9
:1078600000200AE06B00E65A00213000E718FFF71D
:10787000BBFF002802D126800130FEBD017A0198AD
:10788000FFF794FE002802D03B882380F5E70135FE
:10789000EDB2E0E710B5040008880021FFF7A4FF6F
:1078A00003000120002B03D02000197AFFF77EFE91
:1078B00010BD0000054B1B68002B01D1180004E02F
:1078C0009A6852898242F6D1988870470C5FFF1FF0
:1078D000F0B50E27002687B0039302ABFF183E8059
:1078E00005001F4B40891400984207D02B780130C7
:1078F00000976A6880B2FFF78FFE060002212B789E
:1079000018486A68FEF7A2FB00280FD06C89200097
:10791000FFF7D0FF002802D0013C0419A4B2039B5A
:10792000002B00D01C80300007B0F0BD02212B7866
:107930000D486A68FEF78AFB0028E7D102212B7800
:107940000A486A68FEF782FB002807D0002EDED0C6
:107950003B88A342DBD17489013CDFE76C89DEE719
:10796000FFFF0000E6B90011E4B90011E2B900110F
:1079700010B50C00FFF7DEFC03000220002B0AD03C
:10798000002C00D023609B781720FE2B03D00138F9
:10799000FF2B00D1002010BD73B50D0001A904001C
:1079A0001600FFF7E5FF172805D0002E04D12900A7
:1079B0002000FEF727F976BD01221021200000F0FB
:1079C00047FE0028F3D0F6E7014B18607047C04629
:1079D0001C5FFF1F37B56B469D1D0100040002228E
:1079E000280003F0B5FE2B88B02B0ED12379122B83
:1079F00009D12300FA331B78012B06D101216088BD
:107A000000F0E0F801E01B2BF8D037BD10B5054BB6
:107A10000421187000F098F8FFF74CFDFEF770FB9A
:107A200010BDC046205FFF1F0020F0B50BB20F0055
:107A300087B0834234DA274B187803F0E1FD051E46
:107A40002BD00378A02B25D103AE3100FEF7E4F84C
:107A5000041E0BD1B378DB0724D51F4B06341B68FB
:107A6000002B03D03100688898470400A8680028DC
:107A700001D003F045FD002C08D1184A039B1340A8
:107A8000174A934206D0B3781B2B03D00121688894
:107A900000F098F8280003F013FE802000027840E0
:107AA00007B0F0BD0F4B1B68002B10D03100688869
:107AB0009847041EDAD07378002BD7D1B27801A989
:107AC0000A704B800C716888FDF7F6FFCEE706243C
:107AD000F1E7C046205FFF1F185FFF1F00FFFF0098
:107AE000000112001C5FFF1FF7B50190FC200D0084
:107AF00017001E0003F0CCFD04001320002C12D050
:107B0000B02320002370089BF422677065802671E3
:107B10000830002B08D0190003F05AFB210001980F
:107B200003F02EFC0020FEBD089903F069FBF5E789
:107B300010B5041E06D00078FD2803D803F048FED7
:107B4000FF23237010BD00000A1F93B210B504007C
:107B50000220032B05D882400020024BD1529B18F3
:107B60009C7010BD405FFF1F0B8870B5043B040084
:107B70000D000220032B0BD80121200000F04CFD4A
:107B800003001420002B03D02900200000F0DEFBAE
:107B900070BD000007B51300034A00920A000121DE
:107BA00000F02CFC0EBDC046D17D001107B501923E
:107BB00003220092024B0A00122100F049FC0EBD84
:107BC0004F7E001107B56B4601AA11800449D88089
:107BD00008780633012802D1190003F011FC07BD13
:107BE000215FFF1F0C4B10B518700023FF210B4ABB
:107BF0001380138193819380094A538013705172CB
:107C000093819372D174D3821375517703F0A8FBDB
:107C100000F0FCF910BDC046505FFF1F405FFF1F22
:107C2000225FFF1FF0B58DB06B46002003910C2240
:107C30009B5E834200DBB0E05D4B187803F0E0FC14
:107C4000051E00D1A4E00378902B00D09DE006AF84
:107C500001004688380000F013FA79680400002912
:107C600000D19CE03B88052B6ED13B89032B1CD9AE
:107C700005AC200000F0A2F86288172A61D8398983
:107C8000131D994231D17968237804310291D907C3
:107C900038D5607800F08EF9071E06D000230371F6
:107CA0002378012B08D0132B23D0A868002800D1FB
:107CB00078E003F025FC75E06288029909A800F0DD
:107CC000A6F80290380000F08BF909AA2378387AD8
:107CD0000192002231000092029A00F012F938005D
:107CE00000F064F9029B002BDFD0300000F080F937
:107CF000DBE70378032BD8D16288029909A800F04A
:107D0000D6F8DEE7122B13D1029909A800F0B5F8D6
:107D1000021EEAD127498B88002BC6D0887909A991
:107D20002378019161780091310000F0EAF8BCE716
:107D3000002302AA93833000617809AAFFF72AFF83
:107D4000B3E71D4B0993F6E7042B02D09A1F012AD3
:107D5000ABD8184A043B9B00995A0029A5D0D218E9
:107D6000907831003A0000F0AEF800289DD13B88B1
:107D7000042B03D001213000FFF724FF012C04D194
:107D8000A868002801D003F0BBFB280003F098FC92
:107D90008020039B0002434018000DB0F0BD012875
:107DA00000D182E701213000FFF70CFFEDE7C0466C
:107DB000505FFF1F405FFF1F010017000B7803702B
:107DC0004B784370CB788A781B021343438070470B
:107DD0000A88030002700A88120A42700A88012A7F
:107DE00006D14A8882704A88120AC27004207047FD
:107DF00002208242FBD14A8804309A704A88120AD3
:107E0000DA708A881A718A88120A5A71EFE710B5F7
:107E10000400012082420CD94B780A781B021343DC
:107E20002380834206D1CB788A781B021343638078
:107E3000002010BD022BFBD1CB788A781B021343A4
:107E400063804B790A791B021343A380F0E70B8808
:107E500003700B881B0A43704B8883704B881B0A86
:107E6000C3708B8803718B881B0A4371CB88837125
:107E7000CB881B0AC3710820704703000120082A21
:107E800014D14A780878120202431A80CA78887896
:107E9000120202435A804A790879120202439A80F8
:107EA000CA798879120202430020DA80704710B53F
:107EB00004000120022A05D100204B780A781B0219
:107EC0001343238010BDF8B5060010200F001500E5
:107ED00003F0DEFB04000120002C0ED0A0230C22B6
:107EE000290023806780201D002D07D003F070F942
:107EF0002100300003F044FA0020F8BD03F080F9BF
:107F0000F6E7F7B51E00009008AB142017001D78A7
:107F1000019103F0BDFB041E12D0A2230370019B4C
:107F200047704380099B057146710C220830002B75
:107F300007D0190003F04CF92100009803F020FA53
:107F4000F7BD099903F05CF9F6E737B5041E0FD0C9
:107F50004388002B0CD00025C1881323007A1722F8
:107F600001950095FFF7CDFFFF23658063722570B3
:107F700037BD000010B50C4904004A88002A09D01A
:107F80008B89002B05D00020CB8A0222834201D0AE
:107F900010BD012213000A20434300204032C85480
:107FA000C81842800472F3E7225FFF1F002343805A
:107FB00003707047094B00211A0010B55C88002C33
:107FC00006D01C79844203D10A234B43D01810BD3C
:107FD00001310A330329F1D10020F8E7225FFF1FA6
:107FE00010B50400407A03F0F3FBFF23637210BD69
:107FF0007047043010B580B203F0EAF9002803D0CE
:108000000421494203F034FB10BD000070B5002587
:10801000104CA0682580A581A580A84202D003F05D
:108020006FFAA56000250C4C0C4B606D1D80230081
:1080300058331D70A84202D003F062FA656500252E
:108040006068002801D003F05BFA013508340A2D7E
:10805000F6D170BDE85FFF1F8C5FFF1FDC5FFF1F65
:1080600070B5041E09D1054D2880A881A880A86894
:10807000002802D003F044FAAC6070BDE85FFF1F37
:10808000F0B54B8885B00193002343600A79050061
:108090000F00022A00D07BE0CA88032A17D98B6818
:1080A0005E7819783602DC78D8790E4399781B7A95
:1080B00024021B020C43034353495BBA0B80331D5C
:1080C00093421ED1042C04D0631F022B0ED9012031
:1080D00015E0019A4D4B1201D35A002B06D001989E
:1080E000FFF7BEFF4A4A1369013313610421B868E0
:1080F0002E812C80494203F0BBFA6860002005B055
:10810000F0BD434D042C06D0631F022B0FD9EB6842
:108110000133EB60DBE7019A3C4B1201D35A002B91
:1081200005D00198FFF79CFF2B6901332B61374B7A
:1081300030000293019B029A1B01019300230199D5
:108140008C468B52130063449C8003939E81FFF7FF
:1081500050FF039B041E986016D00421B868494262
:1081600003F086FAFA880100043A200003F030F8A0
:108170000199029AFB888A5A043B9B18029A8B52F7
:108180002B6801332B60A2E7AB690133AB619EE73B
:108190001E4B0293019B1E01029BF35A002B2DD014
:1081A00002998C19A068002828D0012A26D1FA88C3
:1081B0009B189BB27352A189994217D39B1AC0187E
:1081C000B96803F005F8029BA289F35A934200D0E4
:1081D0007DE700222B81A3882B80A3686B60029B24
:1081E000F2520B4A53680133536070E7084A9368B0
:1081F000013393600198FFF733FF68E7044A53693E
:1082000001335361F6E7C046525FFF1FE85FFF1F6F
:10821000585FFF1F70B5051E15D10B4C0B4B188016
:10822000230058331870606D002802D003F068F9FD
:108230006565250050356068002801D003F060F9BD
:108240000834AC42F7D170BD8C5FFF1FDC5FFF1FAD
:10825000F0B51700A12285B0920001934243394B3B
:1082600006001B680C009B18D933FF331D78FDF7FF
:1082700041FF0430854204DD3000FDF73BFF043050
:10828000C5B2BD4207D33A0000213000019B03F084
:1082900067FA05B0F0BD2900380003F061F923004A
:1082A000C6B250331E700393019B290063653800EA
:1082B00003F03EFACBB20293002B02D0039B0136AF
:1082C0001E7000262300503303931B78B34204D85A
:1082D000606D002831D10020DBE7029A2800002AD7
:1082E00004D0013B1000B34200D02800F700E7198A
:1082F000387002F0ADFF786000280ED03A7801990E
:1083000002F066FF019A3B780136D3180E4A0193BA
:10831000D369F6B20133D361D4E7039B187060656B
:10832000A74205D1084A1320D36A0133D362B0E7CC
:10833000606803F0E5F80834F2E703F0E1F80023A1
:108340006365C8E73409FF1F585FFF1FF7B50D00CD
:1083500007000421686803F08BF92B89040003707F
:108360002B891B0A43702B8883702B881B0AC370D0
:108370002E8902250436F6B2F42E15D81B4B9F42E7
:1083800014D10C2003F084F91135011E0CD0902378
:1083900003708E3B0371043B4380154B8460C680A1
:1083A000187802F0EDFF00252800FEBD5C237B431A
:1083B000104AD3180093583301931B78002B0FD128
:1083C0000300320038000099FFF742FF019B0500CF
:1083D0001B78002BE8D13800009902F0E9FFE3E7B1
:1083E000054A0725536A01335362DDE7FEFF0000AB
:1083F000505FFF1F8C5FFF1F585FFF1FF0B587B0F6
:10840000009017200F0016000193FFF7F2FD1325CF
:10841000041E19D00C98031E02D00199201D984704
:10842000030AE370052302AAA0700430908127702C
:108430000098667003A993800494FFF787FF051ED8
:1084400002D0200003F05CF8280007B0F0BD000067
:10845000F0B587B01F000CAB1B7803910593012189
:108460000DAB06001C78049200F0D6F81425002805
:1084700021D02000FFF77EFD0135041E1BD01149DD
:10848000059B0A7803700132D2B2131EC68001D157
:1084900001231A000B7022713000049B039900978E
:1084A000FFF7ACFF051E09D1230021000648074A4B
:1084B000093302F095FF280007B0F0BD0023638068
:1084C0002370F8E7545FFF1F4B7F001130750000E9
:1084D000F8B505000E00064C064F2368002B02D0AD
:1084E0003100280098470434BC42F6D1F8BDC0469C
:1084F000F85FFF1F0C60FF1F0123064A5B42538099
:10850000002313715362044A136053609360D36075
:10851000136170470C60FF1FF85FFF1F020000230C
:1085200010B506499C000859002801D1625010BDC1
:108530000133052BF6D11320F9E7C046F85FFF1F82
:10854000034A5388181A434258414042104070472A
:108550000C60FF1FF0B585B002930AAB1F780CAB1F
:108560001B88009008000E0001920393FFF7E8FFBC
:1085700005001120002D1BD10E48FFF7E1FF04007C
:108580001520002C14D006220B99A771E01D02F0D3
:108590001FFE019B30002371029B29006371009B29
:1085A00066802370039B6562E381FFF791FF2800DB
:1085B00005B0F0BDFFFF000010B5FFF7C1FF0400DC
:1085C0000220002C12D060880121FFF781FF606A31
:1085D000002801D003F054F828220021200002F0E6
:1085E0000FFE012300205B426380207110BD00005C
:1085F00030B5074A074C5588010013780020A54282
:1086000004D05B1A59424B415842104030BDC0461D
:108610000C60FF1FFFFF0000084A10B501230C008B
:10862000904208D0FFF78CFF031E04D0037923404B
:108630005A1E9341DBB2180010BDC046FEFF000079
:10864000024B1879431E9841C0B270470C60FF1F5F
:1086500070B504000D001600FFF772FF002804D16A
:108660000D4B9C4200D0143070BD416A0379052047
:10867000002907D012221A40102A02D10520002E0C
:10868000F2D10F20DB06EFD5897E0C20A94289416B
:10869000494249420840E7E7FEFF0000030010B5E9
:1086A000002800D110BD0348034A41889142F9D007
:1086B0009847F7E70C60FF1FFFFF0000002330B56D
:1086C000C45CCD5C6C40D4540133102BF8D130BD68
:1086D0000F23002210B5C45C64002243CA54C25C5C
:1086E000D209013BF7D210BD0200010010B52032C3
:1086F000103102F0D5FE10BDF0B58BB00390102004
:1087000005931700049102F08BFF0090102002F0F7
:1087100087FF009B13240190002B05D000280CD16B
:108720001324009802F0ACFF019B002B02D018002C
:1087300002F0A6FF20000BB0F0BD102002F070FF89
:108740000600102002F06CFF13240500002E00D15B
:10875000AEE0002819D01022002102F051FD3200B5
:108760002900039802F09CFE041E0ED133787F2B63
:1087700051D830000099FFF7ABFF009B1B787F2B8F
:1087800053D801990098FFF7A3FF300002F078FF5B
:10879000002D02D0280002F073FF002CC1D1102060
:1087A00002F03EFF0600102002F03AFF0290002E79
:1087B0007CD0002878D03A000F3223000125121116
:1087C00005D00F333B4015B25A4253411BB26A1ECB
:1087D0001201002B33D0049BD2B298180099029A50
:1087E000FFF76CFF013D10220021300002F008FD70
:1087F000ADB2049F2D017D19AF4242D0002C33D081
:10880000300002F03DFF029B002B00D189E71800E9
:1088100002F036FF85E729003000FFF759FF2800F6
:108820002549009AFFF74AFFA7E729000098FFF7BC
:108830004FFF28002049019AFFF740FFA5E70F21CD
:108840000F4004998A18D9B28F4208D9D15C06A882
:1088500019540133102BF6D1029A0199C0E7791A05
:1088600048424141C901F2E73900300006AAFFF74A
:1088700025FF3200039806A902F012FE103704000B
:10888000BAE7002CBCD13000029906AAFFF716FF08
:10889000320006A9039802F003FE0822040031000A
:1088A000059802F095FCABE71324A9E71324AAE787
:1088B000002800D06EE733E7ECB90011F0B58BB0BB
:1088C0000F0016000225009000283FD0002A3DD05E
:1088D0000B1DDBB21800029302F0A2FE1135041E3C
:1088E00034D0FDF747FD05003A000099201D02F045
:1088F00027FFEBB20393E3702B0CDBB22F0A00933C
:108900006370FFB22B0E2370A7700193FDF72CFD4F
:108910001022010006A802F013FF2100029A04AB06
:1089200006A8FFF7E9FE051E0DD1039B0822337050
:10893000009B04A9B370019B7770F370301D02F0A7
:10894000FFFEFDF71DFD200002F09AFE28000BB08F
:10895000F0BDF0B58FB00D00149E03900492059306
:10896000002A03D1022420000FB0F0BD002EF9D060
:108970000398FFF7E5FD1424071EF4D072783378CE
:1089800012021A43B3781B041343F27812061A43F7
:10899000036A0192934201D30133E3D1002D03D046
:1089A0003B7901249B07DED50822002106A802F0AE
:1089B00027FC059B13240433DBB21800029302F05A
:1089C0002FFE051ECFD0059A0499043002F0B8FEA0
:1089D00004223100280002F0B3FE390010221031C9
:1089E0000AA802F0ADFE2900029A06AB0AA8FFF71A
:1089F00083FE041E0FD1082206A908A802F0A0FEDB
:108A00000822311D08A802F03BFD012807D1019979
:108A10000398FDF7C9FC280002F032FEA3E7012409
:108A2000F9E7000070B51C4C05002368181E10D033
:108A3000002D14D11A78002A0CD1981C083202F0AB
:108A4000C7FB02F0C5FD0135002808D123681D7061
:108A5000012070BD0A331800082202F0B9FB236818
:108A6000002BF5D0122002F013FE061E0DD0C123FC
:108A700021680370457002311022023002F0A8FB19
:108A800023683100587802F07BFC206802F0F8FD82
:108A900000232360DCE7C0463460FF1FF8B5040004
:108AA0002020FDF755FB0D4EA700BB590500002BFC
:108AB0000DD000280BD0D878FF2809D108492A000A
:108AC0000C55F35907480333611802F089FCF8BDCF
:108AD000290002F0EDFC0028F0D1F8E75060FF1FFC
:108AE0003860FF1FF59C001170B5064D8400635976
:108AF000002B05D0D87802F06BFEFF226359DA70A4
:108B000070BDC0465060FF1F70B506008CB00C00F1
:108B1000150000213022684602F072FB310010225D
:108B2000684602F00DFE1D2021000322684402F079
:108B300007FE6846FFF7D8FD2D2104000322280018
:108B4000694402F0FDFD20000CB070BDF0B50700D7
:108B5000160097B001931CAB1D7830221EAB00911C
:108B60000AA800211C7802F04BFB102239000AA849
:108B700002F0E6FD1022002102A802F041FB0722CC
:108B8000310002A802F0DCFD072202AB9818631E38
:108B90009C41019902F0D4FD02AB9C732B005A1E3C
:108BA000934102AAD3730021102206A802F028FBE9
:108BB00006221D9907A802F0C3FD1A2002ABC018B7
:108BC00006221F9902F0BCFD102200990EA802F0A7
:108BD000B7FD102202AB0EA908781C78013A60405C
:108BE000D2B2087001330131002AF5D10AA8FFF78B
:108BF0007BFD102212A904000EA802F0E9FA10224F
:108C000006AB0EA908781D78013A6840D2B2087008
:108C100001330131002AF5D10AA8FFF765FD0443AD
:108C200010222098E4B212A902F08AFD200017B0A9
:108C3000F0BD70B50E0014008CB001001022684623
:108C40001D0002F07DFD3100082204A802F078FD2D
:108C50002100082206A802F073FD6846FFF744FDD4
:108C600004001022280008A902F06AFD20000CB0C0
:108C700070BDF8B506000D0000243719AC4200D3D2
:108C8000F8BD02F025FC030A3B70631CDBB2013720
:108C90009D4203D90234F054E4B2EEE71C00EDE744
:108CA00073B506000C000225002819D0002917D042
:108CB000032101A8FFF7DDFF6B469A793F231A4095
:108CC000013313436A463000937101A92200FFF774
:108CD0001BFF051E04D10322E01C01A902F078FA53
:108CE000280076BD03785807DA08C00FD20080004C
:108CF0009B0710439B0F1843C0B2704707230B40DC
:108D0000C908C9000B4303707047000070B5040028
:108D1000FFF7EAFE134DA4006359002B21D0186A17
:108D2000002801D002F0ACFC2B59986E002801D02D
:108D300002F0A6FC2B59D86E002801D002F0A0FC4E
:108D40002B59186F002801D002F09AFC2B59586F4C
:108D5000002801D002F094FC285902F091FC002375
:108D60002B5170BD5060FF1F0E4B8000C35870B573
:108D70000C00002B0FD09D68002D0CD02B78201DEF
:108D80000B706B784B70A97CFFF7B8FF2B7E2372BA
:108D90006B69E36070BD10220021200002F030FA00
:108DA000F8E7C0465060FF1F014B18607047C0468F
:108DB0004C60FF1F074A03008000825810B5002A4C
:108DC00006D0D088984203D1012901D1FFF79EFF38
:108DD00010BDC0465060FF1FF0B5264E95B087000D
:108DE0000B93BB590500099112200A92002B31D038
:108DF000D888FFF7A5FB04001420002C2AD02800F7
:108E000010A9FFF7B1FFBB591E781D6A002E23D0B1
:108E10000895FDF7EFFA07000020FDF7F1FA07903B
:108E2000A379E61D069310AD0CA9089800F0E2FAAC
:108E30000EA9280000F0D7FA0B9B0A990493069B11
:108E400009980293079B0396019300970EAB0CAA17
:108E5000FFF77CFE15B0F0BDFDF7CCFA06903000B0
:108E6000FDF7CEFAE31DA779079310AB0600089330
:108E7000DAE7C0465060FF1F30B50C4C85002A5918
:108E8000030085B00120002A0ED018006946FFF7C4
:108E90006BFF2B591A78D888054B002A00D1054B57
:108EA0006A46072100F0D9FB05B030BD5060FF1FB6
:108EB000E7930011F593001130B5094C850029594D
:108EC00085B010226846253102F082F92A59112115
:108ED000044BD0886A4600F0C0FB05B030BDC046E8
:108EE0005060FF1F9194001130B5094C850029593D
:108EF00085B010226846353102F06AF92A591121ED
:108F0000044BD0886A4600F0A8FB05B030BDC046CF
:108F10005060FF1FCF940011F7B54D4F8600102011
:108F2000F4590D0002F07CFBF3592062186A1322F9
:108F300000286CD0033A29009C6802F049F9F359E3
:108F40001A780192002A58D11E6A227D317B9446FC
:108F500051400122019F114201D167461740217DF6
:108F6000914339432175377B4F40BC46604600270B
:108F7000800701D44F081740012102208F40227D35
:108F800082433A432275377B5740BC4660460027F0
:108F9000400701D497080F400420227DBF00824380
:108FA0003A432275627D002794466046727B4240B8
:108FB0000A4201D167460F400121627D8A433A434C
:108FC0006275777B5740BC4660460027800701D416
:108FD00057080F400220627D7F0082431743677568
:108FE000767B00227E40760701D4BA080A40042628
:108FF000617D9200B1430A4362756A78002A08D005
:109000006278002A05D005220533DA7700221000A5
:10901000FEBD04222979114205D1A17C114202D161
:109020000533033AF1E7019A21782C78002A02D11E
:109030000A002100140018220429E8D8042CE6D8DC
:1090400005206043034A05331218525CDDE7C04631
:109050005060FF1FFCB9001110B50A001121024B2E
:1090600000F0FBFA10BDC0462B9500110B0030B587
:1090700087B001AD2B806B4604001100981D0822BB
:1090800002F0A6F82A000B212000024B00F0E5FABE
:1090900007B030BD5395001110B50A001121024BE5
:1090A00000F0DBFA10BDC046A795001113B50B0008
:1090B00011006A4613706B4604000622581C02F029
:1090C00087F86A4608212000014B00F0C6FA13BD5C
:1090D000C795001110B50A001121024B00F0BDFA2E
:1090E00010BDC046179600117FB505000B4BAA00B6
:1090F000D4580800002C0FD0666F237FE2882178B7
:109100000396266F0296E66E0196A46E0094FDF714
:1091100009FC2800FFF7FAFD7FBDC0465060FF1F25
:1091200010B51721FFF7E0FF10BD000070B50A0071
:109130000D00064B0221040000F08FFA060029788A
:109140002000FFF7D1FF300070BDC046F79400113A
:1091500070B586B000236A461370836804001D78DA
:10916000681E0A2859D801A902F082F90606333789
:109170003B3F43474B4F5300180000F042F9062392
:1091800012284BD000281BD16088FFF7D9F908239B
:10919000002813D04279002A47D1264B1A7807239A
:1091A00012070BD5244B1A680723002A06D016682D
:1091B000002E03D0290001AAB04703006A461370AD
:1091C0006B461B786088002B2AD1FFF767FC06B03E
:1091D00070BD180000F06CF9D4E7180000F087F9B2
:1091E000D0E7180000F093F9CCE7180000F0ADF9D3
:1091F000C8E7180000F0C3F9C4E7180000F0F6F95A
:10920000C0E7180000F0F6F9BCE7180000F013FA08
:10921000B8E7180000F013FAB4E707236A461370A2
:1092200069466088FFF782FFD1E70523012AC5D18F
:10923000024BB8E7DD5EFF1F4860FF1F4C60FF1F59
:10924000F8B52C4F8600F35904000D00002B40D0D8
:10925000DA8882423DD15A78062A33D11A78002A18
:109260002ED0012099681A6A097D014206D0157B2B
:10927000054203D007225A700120F8BD02200142A6
:1092800004D0157B054201D00922F4E704200142F5
:1092900004D0127B024201D00B22ECE7164B1B6874
:1092A000002BE9D05B68002BE6D020009847BB5923
:1092B00000215B78122BDFD12000FFF715FFDBE7E1
:1092C0000E4BECE7112A04D1002900D032252900E9
:1092D000F2E7002D08D12000FFF732F9002803D073
:1092E000102302791343037121002800FDF798FA37
:1092F000C2E7C0465060FF1F4860FF1F4C60FF1F61
:1093000070B50E4E8500AB590400002B13D01B78AE
:10931000002B11D10A4B1B68002B04D05B68002B7B
:1093200001D02000984773595B78122B03D100219C
:109330002000FFF7D9FE70BD024BECE75060FF1F25
:109340004C60FF1F4860FF1F094B8000C35810206E
:10935000002B0CD01A6A002A09D09B68002B06D07B
:10936000127A1B7E101C9A4200D9181CC0B270479A
:109370005060FF1F70B503000D0014000220002A8A
:1093800030D000292ED013700B78081D53704B7805
:109390009370FFF7A7FCE070012002212B7A237164
:1093A0006B7B034063716A7B0A4013430422637141
:1093B0006E7B1640334363716E7BF608F6003343D1
:1093C00063712B7B0340A371287B014000200B437A
:1093D000A371297B0A401343A3712A7BD208D200D0
:1093E0001343A37170BD10B50A0001000120FFF7FF
:1093F000C1FF10BD10B50A0001000220FFF7BAFF3F
:1094000010BD70B506000C000220002E30D00029DF
:109410002ED07378201D0B70B3784B70F178FFF766
:109420006DFC01223579257271794B1008001340CB
:10943000934010400343881010408000C908034344
:10944000C9000B436373B1794B100800134093407C
:1094500010400343881002409200C9081343C9001A
:109460000B4321202373FCF773FE854201D21220A7
:1094700070BD2220257AFCF76BFE8542F7D8237851
:109480001820042BF4D86378012BF1D80020EFE7E3
:10949000030010B50220002909D0002B07D00322B9
:1094A000481C0A7019000D3201F092FE002010BD18
:1094B00003000222080010B5002B06D0002904D0BA
:1094C0000E32591C01F084FE0022100010BD030072
:1094D00010B50220002909D0002B07D00422481C17
:1094E0000A7019000C3201F073FE002010BD10B597
:1094F000FFF7DEFF10BD03000220002906D0002B7D
:1095000004D0052200200A701B784B7070470300BE
:109510000220002B08D0002906D05B7800200B70B9
:10952000013B082B00D918307047030010B502200A
:10953000002909D0002B07D00622481C0A70190008
:109540000A3201F045FE002010BD10B5FFF7B0FF54
:1095500010BD02000B00022010B500290ED0002A19
:109560000CD007211970118859701188090A997057
:1095700011180822D81C01F02BFE002010BD03009A
:109580000A00022010B5002B0CD000290AD09978CF
:109590005878090201431180901CD91C082201F05F
:1095A00017FE002010BD030010B50220002909D0CD
:1095B000002B07D00822481C0A701900921801F0ED
:1095C00007FE002010BD02000B00022010B500298C
:1095D0000BD0002A09D00921197011781818597078
:1095E000511C062201F0F4FD002010BD10B5FFF75C
:1095F0005FFF10BD02000B00022010B5002A09D049
:10960000002907D05178197011180622581C01F052
:10961000DFFD002010BD030010B50220002909D095
:10962000002B07D00A22481C0A701900063201F0EC
:10963000CFFD002010BD10B5FFF73AFF10BD0200AE
:109640000B00022010B5002A06D0002904D0180013
:109650005178FFF753FB002010BDF0B585B017001F
:109660001E006A4606230500080091819380FEF7DC
:10967000C0FC1324011E02900CD03800B047041E19
:1096800005D1280001A9FEF76FFA041E02D0029846
:1096900001F036FF2800FFF701FA200005B0F0BD09
:1096A000F0B504008BB0019115000021102202A832
:1096B00001F0A6FD334EA700B85900283CD0C3885E
:1096C000A34239D10378002B36D14278062A18D12B
:1096D00002000100553235310C3006ABFFF7A9FA14
:1096E000002829D12000FFF72FFE020006A902A8BA
:1096F00001F06EFD200002A902F012F801200BB06B
:10970000F0BD816E002917D00B8A112A28D19D4205
:109710000ED101981231093A01F0B2FE012807D1A9
:10972000BB5920009D6EFFF70FFE29000200DEE707
:1097300032212000FFF7D8FC2000FEF701FF061EB3
:109740001BD0416A002918D00B8AAB4215D10822E0
:109750000198123101F094FE01280ED1716A0AE0DD
:109760009D42E9D108220198123101F089FE0128B9
:10977000E2D1BB59996E8A7EB9E7200001F060FE04
:10978000BCE7C0465060FF1FF0B56B4D87007E59A7
:1097900085B0337802900393002B00D087E0B36844
:1097A000346A01937078062817D101221B7D134279
:1097B00002D0217B114218D10222134202D0217B18
:1097C000114251D10422134203D0237B134200D013
:1097D0008BE0019B5A7DEB5991E007380428F8D8BB
:1097E00001F046FE032E42678300B36E002B03D1C7
:1097F0001C2001F015FFB066EB599C6E002C1CD0AC
:1098000010220021200001F0FBFC0298FFF79CFDD4
:1098100001002000FFF72DFA01F05AFE20822000FF
:1098200008211230FFF725FA0298FFF78DFDA07688
:10983000EB592100D888FFF70FFC0822EB591CE0F8
:10984000B36E002B05D01A00198AF0881232FFF788
:109850000DFC0222019B197DEB5911423DD0207B6A
:1098600010423AD0073208E0F488FCF7DBFD010033
:109870002000FFF711FC0A22EB595A70029B9C0052
:109880002A595378073B042B11D8D088FEF758FE8D
:1098900000284ED0C3895A08D2182849029B029842
:1098A000CB542B5941180433254801F099FD05B0DC
:1098B000F0BDFCF79FFD03000120834201D1002091
:1098C0000393EB59DE88FCF79BFD039902003000FF
:1098D000FFF7ECFB019AEB59117D042211420CD0E9
:1098E000217B114209D00B22C7E7F688FCF73CFD2B
:1098F00001003000FFF7EEFB6BE7019A527D01217A
:109900000A4204D0607B084201D00C22B5E7022154
:109910000A4204D0607B084201D00E22ADE7042148
:109920000A4204D0627B0A4201D01022A5E712222B
:10993000A3E7FA225200B0E75060FF1F5460FF1FF8
:10994000FF9C001110B5064B1A7804231000184034
:109950001A4200D00348FFF727FA002010BDC04686
:10996000DD5EFF1FA43DFF1F70B50400FFF7D4FAB2
:10997000051E43D12000FFF77FFA234EA400A05913
:109980008268937CDB0708D50321036A1B790B40AF
:10999000012B02D1017F0B430377431DD97F8B1E1F
:1099A000022B0DD8022900D00121C088FCF790FFBE
:1099B000042133591A7F59700A431A77280070BD61
:1099C00001290CD102231022437000210C3001F038
:1099D00017FC305910213530FFF74BF9EEE7052918
:1099E000ECD10223D118437010220C3001F0F0FBAF
:1099F00004233259117F0B431377EAE7082518280F
:109A0000DCD1053DDAE7C0465060FF1FF0B58BB0F2
:109A1000059143887E4F9E00F45915000493002C55
:109A200015D1012902D000200BB0F0BD101D5778D0
:109A30001678FFF757F9EB68320002932B7A0499F6
:109A4000019300903B002000FCF70CFFEBE7E3885C
:109A5000049A934201D00820E6E72378012B00D135
:109A6000D4E0059B581E092800D9CFE001F000FD85
:109A700005CE0A29CC506C859AB229000498FFF7CC
:109A800073FFD1E7200029001022453001F0A0FB30
:109A9000B9594B78042B02D1013B4B70C3E70B0043
:109AA0000A00253335320C310498FFF795F90498F4
:109AB000FFF702FA0522431E9841BB59C0005A70B5
:109AC000B2E7200029001022553001F081FB049BF1
:109AD0004F4C9D00295904980A0006AB55320C31B1
:109AE000FFF77AF929591022453106A801F0C8FC80
:109AF000012808D10498FFF7F7F90590002804D150
:109B000006222B595A7005988EE708230593FAE729
:109B100063780C2B7AD1E36E002B03D11C2001F06B
:109B20007FFDE066BB59D86E00286FD01022290057
:109B300001F04EFBBB590498DC6EFFF705FC0D22CB
:109B4000A076BB595A706EE7E06E00285ED063784D
:109B50000D2B5BD12B8808220382A91C123001F047
:109B600037FBBB599A68517D0222114226D0186AF0
:109B7000407B104222D00C32E4E763780E2B45D1B3
:109B8000236F002B03D1162001F04AFD2067BB593B
:109B9000186F002803D01022290001F019FB0F22B2
:109BA000BB59CFE763780F2B30D1206F0622691C99
:109BB000103001F00DFBBB599A68517D042211420F
:109BC00003D0196A497B1142D5D100210498FFF7CF
:109BD0008BFA28E7636F002B0DD0BB59586F002814
:109BE000F3D01022290001F0F3FA0122BB595242AE
:109BF0005B6F1A61E9E7142001F012FDBB59606741
:109C00005B6F002BE9D126E72978DFE707200BE718
:109C10005060FF1F10B5064C207001F021FD062199
:109C20002078FDF791FF0348FEF778FC10BDC04691
:109C30006360FF1FB58D001100200BB270B50D00E1
:109C4000834216DA264B187801F0DAFC041E0DD098
:109C50000378922B0ED0A02B37D0224B1878FF28F8
:109C60003AD0210001F08CFB002835D18020000281
:109C7000684070BD43780E2B0BD03E2BEDD183781E
:109C8000052B12D0082BE8D181798088FFF7D8FA0C
:109C900008E0154B82889A42DFD183681878591CF6
:109CA000FEF7C0FE002817D1D7E7104B1B785B07E3
:109CB00012D50F4B1B68002B0ED09B68002B0BD0CE
:109CC000C289811D80889847ECE7FFF741FAA068B8
:109CD000002801D001F014FC200001F0F1FCC5E7E0
:109CE0006360FF1F9D3DFF1F18200000DD5EFF1F0A
:109CF0004C60FF1F10B50078FFF712FA10BD10B5C9
:109D00000078FFF7FDFA10BD0C234343084A10B555
:109D10009B185A68002A03D0012901D1904710BD31
:109D20009B68002BFBD00029F9D19847F7E7C04684
:109D30008060FF1F01238340094A10B5946B1C43C8
:109D40009463506B98435063D46B2000984301296F
:109D500001D120001843D063116B0B43136310BD76
:109D600000800040F0B500240127154B85B0DA6B68
:109D7000144E03921A6C0192DA64019BE3403B4259
:109D800017D0039DE5403D400295E5B202992800B9
:109D9000FFF7BAFF316A736A002908D03900002B37
:109DA00001D0029979402800FFF7C4FF01E0002BA1
:109DB000F9D101340C36172CDFD105B0F0BDC04607
:109DC000008000406460FF1F064B01215A68C240BA
:109DD0000A4204D01B68C3401800084070471B6D3E
:109DE000F9E7C046008000400122064B824000296E
:109DF00003D0D9680A43DA607047D9689143D960C3
:109E0000FAE7C0460038004030B5032444430F4B06
:109E1000E25C1B199C785D7801232D1B0135AB405A
:109E2000013BA340A140DB430C00122807D808499E
:109E300092005218116819402143116030BD054A43
:109E400011680B4023431360F8E7C04643BA001182
:109E500008F0004014F00040C21F70B5D4B20623D1
:109E6000092C0BD80125084C9540002908D0002169
:109E7000FFF7CAFF23682B4323600023180070BD3F
:109E80002368AB43F8E7C04600380040214BF0B5EB
:109E90001B185B78022B21D1032444431E4A1F4E1A
:109EA000A35C12199478012215008540B76B013C20
:109EB000E4B23D43A240B563194C122815D89B006B
:109EC00000290CD117495B1899680A439A6001234D
:109ED000205C154A834011680B431360F0BD1149A3
:109EE0005B18996891439960F1E70E4B00290DD1F9
:109EF00059690A435A61225C1328E8D00123203AA9
:109F000093400A49086803430B60E7E759699143A6
:109F10005961F0E76460FF1F43BA00110080004000
:109F200088BA001100F00040A0F00040A4F000400A
:109F3000F8B500241B4E1C4D1C4B1B5D012B1FD183
:109F4000194A9269E2401A420BD00122B25693405C
:109F50002200143AD2B2022A09D815494A69134399
:109F60004B61013402360C35172CE5D1F8BD0022C7
:109F7000B2560F499200521891680B439360F0E774
:109F8000022BEED1E7B23800FFF71EFF0123584045
:109F9000C1B23800FFF77AFF3800FFF715FF687786
:109FA000DFE7C04615BA00116460FF1F6560FF1F40
:109FB00000F00040012202388240054B002903D006
:109FC00059690A435A617047596991435961FAE7DF
:109FD00000380040F8B50E0001210F008740114AFB
:109FE0000400D368FD43BB43D360831E8B4201D87A
:109FF000FFF7E0FF00212000FFF72EFF0A4A0B4B7E
:10A000005168012E05D139431B1951605E70002043
:10A01000F8BD2940516002221C1962709A691540EE
:10A020009D61F4E700380040008000406460FF1F3D
:10A03000012210B58240074B002906D019680A4357
:10A040001A600121FFF7C6FF10BD1968914319601E
:10A05000F7E7C046008000400C2370B5002543435D
:10A060000A4A29009B181D70094B04001B185D70DB
:10A07000FFF7B0FF0123A340064928000A681A43EE
:10A080000A6005490A689A430A6070BD8060FF1F34
:10A090006460FF1F348000403080004070B50400D1
:10A0A0000E00FF2813D003250540FFF7D5FF084A0F
:10A0B000A3089B009B183F22ED00AA40AE40196800
:10A0C00020009143314319600121FFF78DFE70BDDF
:10A0D00018380040F8B50C244443134B0500E4182D
:10A0E0006368002B03D1A3681220002B1AD0022230
:10A0F00001270E4B00215B195A7028002770FFF7CB
:10A1000069FF63681E1E08D0A3683E00002B04D0C0
:10A110002800FFF759FE4640F6B228003100FFF74D
:10A1200009FE0020F8BDC0468060FF1F6460FF1F6D
:10A13000F7B5C420FF222B4B80001958002491430F
:10A140003F3A0A431A508022274F5202274E1A6084
:10A15000274B1D5D002D21D0A31E012B03D801210B
:10A16000E0B2FFF727FF012D18D11F4B9B69E34099
:10A170002B4213D0E3B218000193FFF725FE010034
:10A180000198FFF755FFE3B2143B022B1DD80121C4
:10A190007156184A8D405369AB4353613B7F002B86
:10A1A0000DD0E5B22800FFF795FF2800FFF70CFE61
:10A1B0007B7F0100834202D02800FFF7A5FD013418
:10A1C0000C370236172CC3D1F7BD0121002371567D
:10A1D000F3568D40074A9B009B189A68AA439A60E1
:10A1E000DCE7C04600E100E06460FF1F15BA001123
:10A1F0006560FF1F00F0004010B501210400FFF76B
:10A20000E9FE0123044A002011194B70A340916913
:10A210000B43936110BDC0466460FF1F70B50E0014
:10A2200015000400FFF718FF0C236343094A2000C0
:10A230009B189D605E60FFF74DFFF021064B074ABB
:10A240008900051E5A5002D02000FFF705FF2800A4
:10A2500070BDC0468060FF1F0000FF1F659D00119C
:10A2600070B5134D07202C78002C1FD198222100A7
:10A270005200280001F044F80123C420FF222B7073
:10A280000C4B80001C635C630B4B1C605C600B4BD5
:10A29000195891433F3A0A431A50802252021A60D9
:10A2A0000D20074A074900F0DBFF200070BDC046C3
:10A2B0006460FF1F00800040A0F0004000E100E06B
:10A2C00031A10011319F001170B51D0002240C292D
:10A2D00010D8094ACA40D2070CD5FBF745FF041E27
:10A2E00008D1059A04992800FBF75AFFFCF7C8FD2E
:10A2F000FFF728FB200070BD1210000030B50D786C
:10A3000002232C009C43184201D02B431C0008253B
:10A310002300AB43284201D02B00234320241D00FF
:10A32000A543204201D01C4325002A230D7018426A
:10A3300004D011781E3B0B43137030BD0028FCD1B4
:10A340000C2113788B43F7E7F8B51D0006AB1B888B
:10A35000140007AA0E000B201778002B27D10A78CB
:10A36000022A49D14A68507811780002244A0843E9
:10A370008018042840D801F07BF803121D1B23002D
:10A38000F06800F0E5FF021CC0B2B84200D93A1CE8
:10A39000D2B22000F1682A8000F01AFF06E0022203
:10A3A000F3681B882A8023701B0A63700020F8BDA5
:10A3B0000622EEE701232B80F3681B782370F5E774
:10A3C000F368002B16D008222A801A8822701A8877
:10A3D000120A62705A88A2705A88120AE2709A8829
:10A3E00022719A88120A6271DA88A271DB881B0ACC
:10A3F000E371DBE72B80D9E701202B80D7E7C0464C
:10A4000000D6FFFFF7B516000A781D0008AB1F88BD
:10A410000C000123022A18D14A68507811780002F2
:10A420002B4A0843801803280FD801F021F8022591
:10A430004439E06800F08CFFC0B20723B84204D36F
:10A440007B190193152B02DD0D231800FEBDE0687A
:10A450002A003100C01900F0BBFE6B4600209B882B
:10A46000E268D0541B4B1B68834203D01B688342B5
:10A4700000D098470023E8E70B23002FE5D1022DF9
:10A48000E2D1737832781B021343E2681380114BD8
:10A490001B68002BEED01B68002BEBD00120E8E7F7
:10A4A0000B23002FD1D1062DCED12A003100E06838
:10A4B00000F08EFEDEE70B23002FC6D1012DC3D1A5
:10A4C00032787533012AC0D8E3681A70D2E7C046E3
:10A4D00000D6FFFF7062FF1F70B50C001500072843
:10A4E00037D800F0C5FF041436361B36242E18204A
:10A4F00015290BD8184E16220021300000F080FEDE
:10A5000022002900300000F063FE002070BD1820FA
:10A510000229FBD11288114B1A80F6E7182008296E
:10A52000F4D10A000E48290001F012F9EDE71820D5
:10A530000129EBD10B4B10780B49DA69FFF7DEFEEE
:10A54000E3E718200129E1D1064B10780749DA6BBF
:10A55000F4E70220DAE7C0465862FF1F463EFF1FBD
:10A560003C3EFF1FCC3DFF1FF43DFF1F143EFF1F6D
:10A57000030010B50020DB0704D50721024A034879
:10A5800000F08CF810BDC046A0BA0011CC3DFF1FF2
:10A59000054A03001068002803D082889A4201D13E
:10A5A000806870470068F6E76864FF1F0A88030048
:10A5B00008009A4204D08A8804309A4200D00020D1
:10A5C00070470000F8B5F22200230D4F0D4E796858
:10A5D000050042433370994200D07B600A4C002151
:10A5E000200000F00DFE00231A007C60AB4202D177
:10A5F00000203370F8BD01332280DBB2F234F5E77E
:10A600006065FF1F5E65FF1F6C64FF1F73B56B46BF
:10A6100001900600684615001980FCF763FF041ED0
:10A6200011D1002D0FD07689002E11D00C2000F012
:10A63000F7FF00280ED0084A046013688680856002
:10A64000002B02D11060200076BD1A001B68F7E7CE
:10A650000224F8E71324F6E76864FF1F01210022B3
:10A660000A4B10B549420A4C198099809A719A7028
:10A67000084B2070012019805A60FFF7A3FF207853
:10A68000FCF78EFF0448FDF749FF10BD7862FF1FFD
:10A690006865FF1F6065FF1F49A70011022310B501
:10A6A000002802D0FFF7B2FF0300180010BD000021
:10A6B000030010B50020DB0704D50421024A03483B
:10A6C000FFF7A4FF10BDC046B4BA00114C3EFF1FF7
:10A6D000F0B50E2687B003930CAB1F8802ABF618BB
:10A6E0000500080031000292FDF77EF80400012009
:10A6F000002C0FD03088FFF74BFF03000E20002BFB
:10A7000008D05E68002E05D021002800039B029A25
:10A710000097B04707B0F0BD0A4B10B5984207D17B
:10A720000122002352420A808B708A808B7110BDF7
:10A73000FFF73CFF0028FAD001235B42038000238F
:10A740008370F4E7FFFF0000F8B5050001290AD186
:10A75000134E00243388F227AB4219D02800114948
:10A76000FFF7DAFF06E0022904D10139FDF754FFB3
:10A770000028EDD0F8BD3B0063437268D018D35A6F
:10A78000002B09D03A00002100F03AFD0134E4B278
:10A79000054B1B78A342EED801235B423380DDE7F3
:10A7A0006065FF1F7862FF1F5E65FF1F10B5FFF732
:10A7B000FDFE03000020834200D0987810BD000009
:10A7C000F0B589B01C000EAB80CB03901E8810AB97
:10A7D0001B78049202930B7A0D00DB0616D42B78BB
:10A7E0000593022B24D00498FFF7D2FE002812D044
:10A7F00003689C46002B0ED0029B22000193290087
:10A800003B00644603980096A04705E00498FFF7D4
:10A81000BFFE002802D10E2009B0F0BD8368002BD6
:10A82000F9D00A222900039898470028D7D0F3E7E7
:10A830006B6858781A786B4B000210439842D2D854
:10A84000043B984210D2684B984242D015D8674BCF
:10A85000C0180128C7D80B20002EDDD1EB681A786C
:10A8600059683A80200028E0614BC018032800D9BD
:10A8700079E000F0FDFD846A789E5E4B9842B2D18B
:10A880000B20002EC8D101233B80EB6831001B78E0
:10A8900023706889013080B2FCF7A6FF3A88031E56
:10A8A0000ED0017802328A183A8042896270428959
:10A8B000120AA27059680278E01C00F089FC06E0D8
:10A8C00004323A8031000422601C00F099FC002020
:10A8D000A2E70B20002E9FD1EB6807A91E88042356
:10A8E0003B80330A300026706370FCF77DFF051E45
:10A8F00028D004AB9A890E2304A95B183E49C66888
:10A90000FCF7E6FF00280BD12B783C486A680599D4
:10A91000FBF79CFB002803D1012304AA5B42D381EF
:10A920003278022A06D17168201D00F051FC3B8864
:10A9300002333B800E2304AA9B181B88A3701B0ABA
:10A94000E370C4E704ABDE81F4E70B20002E00D0F7
:10A9500062E7E9680398FFF729FF02233B80207034
:10A96000000A6070B3E70B20002E00D054E70222EB
:10A97000EB681B883A8023701B0A6370A7E7E868BE
:10A9800000F0E6FCC2B203000720B24200D243E767
:10A990000DD00299DBB27118994202DB921BD3B23F
:10A9A0000293029BE9681A003B8089195AE7002349
:10A9B000F6E70B20002E00D02EE70722EB683A8046
:10A9C0001A7822705A7862705A88A2705A88120ACD
:10A9D000E2701A792271DA886271DB881B0AA3712E
:10A9E00075E7C046042900000228000000D8FFFFD8
:10A9F000FFD6FFFF03280000FFFF0000E4B90011AD
:10AA0000F0B58DB06B460020089120229B5E8342FA
:10AA10003DDAA64B187800F0F3FD071E32D003781C
:10AA2000B02B2CD10079023816281FD800F088FDF1
:10AA300017001E001E001E0031001E0096001E00A2
:10AA40001D011E0052011E0073011E00CD011E00DB
:10AA500050021E001E001E008E021E00E302944BD8
:10AA600094491B8878880B80FBF730F83800FCF796
:10AA7000B1FF914B1B68002B01D03800984738007C
:10AA800000F01EFE8020089B0002434018000DB01D
:10AA9000F0BDEE220021874800F0B2FB0BAA3B7B01
:10AAA0007989388900923A000D32FCF7B5FD04002F
:10AAB000804B1B78002C3FD146E0804B7888059373
:10AAC0007F4B4100CB5A0BAE073BDBB2328802937F
:10AAD000002301937B4B210006930093059BFFF716
:10AAE0006FFE744D002810D1069B3A8A1B889A424B
:10AAF0000BD138000599123000F0C2FC002804D0B8
:10AB00002B7862899B00EB185A80162306A81B1825
:10AB1000328820007989FCF7DBFE2B7804009A004C
:10AB2000AA1851880029C3D00133DBB22B7000284A
:10AB300007D006A9C98A9180634A12889A42BCD874
:10AB400002E0012149429180002B04D059497888C4
:10AB5000FAF7F0FF8AE73E890A2479E000253E896A
:10AB6000574B06937B88069A5B009B5A033B9D429A
:10AB700002DB002DF0D05BE0162206A812183B7B0A
:10AB8000798900923A0030000D32FCF745FD0590BE
:10AB9000002858D04689017A7888FCF707FD041E02
:10ABA00044D1464B78880793069B4100C95A454BD0
:10ABB0000439C9B206AAD28A06930291019400937D
:10ABC0000599079BFFF7FCFD041E2FD1069B394911
:10ABD0001A88931C002D26D14B807988384B490068
:10ABE000CB5A5119033B8B4220DD059B31485B89D1
:10ABF00041190B71A91C0135C9B2EDB20591451976
:10AC00001B0A2B71059B2D490433181800F0E0FA3C
:10AC10002C4B059A1B88D318DDB22C4B9E4205D0D5
:10AC20000136B6B29CE749889942D6D0002D0CD0A7
:10AC3000204C2800618800F0FBFB20702100788800
:10AC4000FAF788FF12E7059CF0E7002C00D183E7B4
:10AC50007B78142B00D109E716493B794E800B70A5
:10AC60000C717888FAF728FF00E7162406ABE41881
:10AC700021003889FCF7B8FD011E00D1B7E17888C2
:10AC800022880F4C45002C5B0A4D013CE4B2029433
:10AC900000240F4B01940095FFF792FD041E00D095
:10ACA00014E129007888FAF765FFDFE66865FF1F81
:10ACB0003C3DFF1F8062FF1F7462FF1F7463FF1F14
:10ACC000B05EFF1F6464FF1F3A3DFF1FFFFF0000DF
:10ACD0008262FF1F162406ABE41821003889FCF7B6
:10ACE00083FD011E00D182E178882288AE4C4500A8
:10ACF0002C5BAE4D013CE4B202947C89AC4B0194D8
:10AD00000095FFF75DFD041E00D0DFE02900788884
:10AD1000FAF73AFFAAE60025A44B1D803B00F63364
:10AD20001B78A24A78880792AB4208D99E4B1288BA
:10AD30000693069943005B5A013B9A4203DB07994D
:10AD4000FAF72CFF92E616246B00FB18059306AB6E
:10AD5000E418059B21001889FCF746FD011E03D16C
:10AD6000059B01241E8973E77888924B2288069CF4
:10AD7000099343001B5B904E013BDBB2029300231F
:10AD800000960193099BFFF71BFD041E02D0059B53
:10AD90001E895DE77B88069A5B009B5A079A10889C
:10ADA00032881218934202DC1B1A013B33807F4C1D
:10ADB000023032880999001900F00AFA2388328893
:10ADC00001359B182380EDB2A8E70BAA3B7B79895C
:10ADD000388900923A000D32FCF71EFC00250590E0
:10ADE000059B002B04D10A24002D00D16EE060E009
:10ADF000059B7888197AFCF7D9FB0100041E63D102
:10AE0000694C6C4B788806940993069B4400E45A7D
:10AE1000694B063CE4B20BAE328807930294019171
:10AE200000930599099BFFF7CBFC041E4CD1079BAF
:10AE30005E491B881A1D002D30D14A80059B5B4C52
:10AE40005A8963191A716B1C9BB2E318120A1A71A2
:10AE5000162306A832881B1879890598FCF738FD57
:10AE6000FF21AA1C2E1D03350B00059092B2B6B22D
:10AE7000ADB2002803D006ABDB8AD9B21B0AA218F8
:10AE8000651911712B714C4D301D2A8849492018C4
:10AE900000F09EF92B88F618B5B2A1E749889142D7
:10AEA00007D17A8806995200525AEB18053A9A420D
:10AEB000C4DC3E4C2800618800F052FB2070210069
:10AEC0007888FAF775FED1E5002DF2D13E89BFE60C
:10AED000162606ABF61831003889FCF785FC3D00D4
:10AEE0000400FA3500282DD0037A9B060CD40022EA
:10AEF0007B893989788800923A000C32FFF7E8FBA9
:10AF0000041E10D03E8915E03088FFF741FB002871
:10AF10001AD08368002B17D0210012227888984716
:10AF2000041EE4D0EEE72B78002B02D17888FAF7E4
:10AF30004FFE00262B78002B00D097E5002C00D187
:10AF400094E585E60124DDE70E24DBE7162506AB54
:10AF5000ED1829003889FCF747FC041E47D0037A16
:10AF60009B0611D4154A7B881188994203D0144856
:10AF7000814207D11380134BF2261D780023D9B2EA
:10AF8000A94221D30924A1E72888FFF701FB002863
:10AF90002FD08368002B2CD021001222788898476C
:10AFA000041EDFD092E7C046B05EFF1F8062FF1F25
:10AFB0008262FF1F7463FF1F6464FF1F6065FF1FD1
:10AFC000FFFF00005E65FF1F3100594354680133E5
:10AFD0006018615A0029D2D13C0008342100F222C5
:10AFE00000F0F6F821007888FAF7FAFD3EE5012432
:10AFF0006CE70E246AE71D4B1A887B889A4231D091
:10B000007888FAF7F7FD31E5F22305985168434354
:10B01000CD18C95A00291FD03B7A012B0BD16C885F
:10B02000AB887888AA1D0094FFF752FB041E02D05B
:10B0300000233B722E88F2220021280000F0E0F865
:10B0400000232B80059B0133DBB20593084B059948
:10B050001B78064A8B42D7D801235B421380002C11
:10B06000CED0F5E5002634000596EFE76065FF1FBA
:10B070005E65FF1F70B504000E001500FFF796FA1D
:10B08000031E08D131000548FFF790FA0300112094
:10B09000002B02D01C8000209D7070BDFFFF0000BF
:10B0A000F8B50B4F06003B780D001400FF2B0ED0B7
:10B0B0000A2000F0EDFA011E09D0B123038000231D
:10B0C00046800371C5800481387800F059F9F8BDD5
:10B0D0008D3EFF1FF7B50F0008A90600088809A9D3
:10B0E0000B240988002821D10234022B1ED1557867
:10B0F00013782D021D432B008B4301937334002BD7
:10B1000014D1FB68300019000093FFF74FFB019C3E
:10B1100085420BD02A0030000099FFF7ABFF041ED8
:10B1200004D12A0030007989FFF7BAFF2000FEBD64
:10B13000F0B50E7885B003900AA805880120022E8C
:10B140000DD14C682778647824023C43054FBC42FB
:10B1500005D10398DBB201960095FFF7BBFF05B060
:10B16000F0BDC04602290000034B10B51B68002B40
:10B1700000D09847FEE7C0466C65FF1F07B501A8E1
:10B18000FFF7F2FF044A05480021121A00F0B8F850
:10B19000F8F730FBFEE7C0467065FF1F903EFF1FCB
:10B1A00001B40248844601BC604700BFE130FF1F84
:10B1B00001B40248844601BC604700BFADAE000048
:10B1C00001B40248844601BC604700BF3D1800003E
:10B1D00001B40248844601BC604700BFE94C01004D
:10B1E00001B40248844601BC604700BF8B52010095
:10B1F00001B40248844601BC604700BF9DA900001D
:10B2000001B40248844601BC604700BF154D0100EF
:10B2100001B40248844601BC604700BF25260000F7
:10B2200001B40248844601BC604700BF3935FF1FA6
:10B2300001B40248844601BC604700BF657101004B
:10B2400001B40248844601BC604700BF056A0000A3
:10B2500001B40248844601BC604700BF017F000082
:10B2600001B40248844601BC604700BF812BFF1F28
:10B2700001B40248844601BC604700BFE12AFF1FB9
:10B2800001B40248844601BC604700BF1D4B010069
:10B2900001B40248844601BC604700BFA533FF1FCC
:10B2A00001B40248844601BC604700BF6D33FF1FF4
:10B2B00001B40248844601BC604700BF455000000D
:10B2C00001B40248844601BC604700BF392BFF1F10
:10B2D00001B40248844601BC604700BF8D120000E3
:10B2E00001B40248844601BC604700BF4D1F000006
:10B2F00001B40248844601BC604700BF212DFF1FF6
:10B3000001B40248844601BC604700BFB70E00008C
:10B3100001B40248844601BC604700BFB14E000042
:10B3200001B40248844601BC604700BF6DBC000008
:10B3300001B40248844601BC604700BF691F000099
:10B3400001B40248844601BC604700BF01240000EC
:10B3500001B40248844601BC604700BFDD520100D1
:10B3600001B40248844601BC604700BF7918000060
:10B3700001B40248844601BC604700BFED4A0100A9
:10B3800001B40248844601BC604700BF594F010028
:10B3900001B40248844601BC604700BF2534FF1F4A
:10B3A00001B40248844601BC604700BF5D1700003D
:10B3B00001B40248844601BC604700BF7D18FF1FEE
:10B3C00001B40248844601BC604700BF6532FF1FDC
:10B3D00001B40248844601BC604700BFE928000070
:10B3E00001B40248844601BC604700BFA946010081
:10B3F00001B40248844601BC604700BFF94C01001B
:10B4000001B40248844601BC604700BFE117000058
:10B4100001B40248844601BC604700BF5952010094
:10B4200001B40248844601BC604700BFB131FF1F30
:10B4300001B40248844601BC604700BF350E0000DD
:10B4400001B40248844601BC604700BF091B0000EC
:10B4500001B40248844601BC604700BF0D520100A0
:10B4600001B40248844601BC604700BF5522000079
:10B4700001B40248844601BC604700BF4D36FF1F3F
:10B4800001B40248844601BC604700BFCD4C0100B6
:10B4900001B40248844601BC604700BFE533FF1F8A
:10B4A00001B40248844601BC604700BFE548000083
:10B4B00001B40248844601BC604700BF5147010007
:10B4C00001B40248844601BC604700BFEDA50000FE
:10B4D00001B40248844601BC604700BF2951010005
:10B4E00001B40248844601BC604700BFC52100008A
:10B4F00001B40248844601BC604700BF212400001B
:10B5000001B40248844601BC604700BFD94901002C
:10B5100001B40248844601BC604700BFF30E00003E
:10B5200001B40248844601BC604700BF792EFF1F6A
:10B5300001B40248844601BC604700BF51250000A9
:10B5400001B40248844601BC604700BF6136FF1F5A
:10B5500001B40248844601BC604700BFA54F01000A
:10B5600001B40248844601BC604700BF090E0000D8
:10B5700001B40248844601BC604700BFBD30FF1FD4
:10B5800001B40248844601BC604700BFC9A900005D
:10B5900001B40248844601BC604700BFB130FF1FC0
:10B5A00001B40248844601BC604700BF156B01002E
:10B5B00001B40248844601BC604700BFE528FF1F74
:10B5C00001B40248844601BC604700BF492DFF1FFB
:10B5D00001B40248844601BC604700BFD91B00008B
:10B5E00001B40248844601BC604700BFB54C01006D
:10B5F00001B40248844601BC604700BF21460100F7
:10B6000001B40248844601BC604700BFF54E01000A
:10B6100001B40248844601BC604700BF75A9000020
:10B6200001B40248844601BC604700BF3D4B0100A5
:10B6300001B40248844601BC604700BF456B01006D
:10B6400001B40248844601BC604700BFC56D0100DB
:10B6500001B40248844601BC604700BF291C0000B9
:10B6600001B40248844601BC604700BFC9260000FF
:10B6700001B40248844601BC604700BF554901003F
:10B6800001B40248844601BC604700BF014C010080
:10B6900001B40248844601BC604700BF1D4D010053
:10B6A00001B40248844601BC604700BF851F00000A
:10B6B00001B40248844601BC604700BFDD6601005A
:10B6C00001B40248844601BC604700BF434D0100FD
:10B6D00001B40248844601BC604700BF055E00001B
:10B6E00001B40248844601BC604700BF8552010096
:10B6F00001B40248844601BC604700BF9134FF1F7B
:10B7000001B40248844601BC604700BF35550000C3
:10B7100001B40248844601BC604700BFF92AFF1FFC
:10B7200001B40248844601BC604700BF311B0000E1
:10B7300001B40248844601BC604700BF090E000006
:10B7400001B40248844601BC604700BF4551010076
:10B7500001B40248844601BC604700BF810E00006E
:10B7600001B40248844601BC604700BF5118FF1F66
:10B7700001B40248844601BC604700BF0D35FF1F7D
:10B7800001B40248844601BC604700BF5933FF1F23
:10B7900001B40248844601BC604700BFC94A0100A9
:10B7A00001B40248844601BC604700BFB3520100A7
:10B7B00001B40248844601BC604700BF3936FF1F10
:10B7C00001B40248844601BC604700BFC51D0000AB
:10B7D00001B40248844601BC604700BF1147010024
:10B7E000000301030200030304020502060207002E
:10B7F000080309030A030B030C000D000E030F03DB
:10B80000100311001303140315031603A93B0011C1
:10B81000DD3B0011000000000200000022B8001112
:10B82000192A0F180A000000F1590000FD24000039
:10B8300041460100257C0011399C00118D700011DA
:10B84000297A00113952001101AA0011B14E0011DC
:10B850009D3D0011CD3E00110000000016160000B5
:10B86000020000006CB80011F4FFF3FFD2FC0000EE
:10B870000D400011000000000000000054757961C7
:10B880000042312E340030303133006769746875FE
:10B89000622E636F6D2F70767678005448423200C6
:10B8A00002000000B4B80011292A282A272A262AD3
:10B8B000252A242A0A180000E20400007102000070
:10B8C00078EC0000744000001027000060F00000D9
:10B8D00006640000204E000000000000050000008B
:10B8E0001F501D00023CB4000001130014000000B2
:10B8F0008102000030313233343536373839414235
:10B9000043444546000000003D5600119156001189
:10B91000000000000200000020B900116F2A6E2A0A
:10B920001A18000001A00000000000006410B71DFC
:10B93000C8206E3BAC30D9269041DC76F4516B6B5D
:10B940005861B24D3C7105502083B8ED44930FF01F
:10B95000E8A3D6D68CB361CBB0C2649BD4D2D386D5
:10B9600078E20AA01CF2BDBDFB349B5F8000008022
:10B9700000100000000000008F5C0011197300111E
:10B98000B35C001121770011375D0011F7760011CB
:10B99000AD5D0011CD760011FF5D001195780011AD
:10B9A000675E001195780011995E00114F780011C3
:10B9B000AD5D001185760011255E00112D78001116
:10B9C00000000000000000000B5F00112D78001146
:10B9D0006D5F001131730011052A042A012A002A23
:10B9E000022903280128002801180018000000007F
:10B9F00000000000000000000000008701010201BB
:10BA0000020101020102030304010301010101011A
:10BA10000303020103000D000E00100011001300CB
:10BA20001401070108010A010B011C011D02040297
:10BA300005020702080219021A021C021D03010373
:10BA4000020317000201000504000807000B0A00AA
:10BA50001716001D1C010201010504010E0D011144
:10BA600010011413011716011A19020201020B0A20
:10BA7000020E0D021110021413021716030504031F
:10BA80000807030B0A030E0D0001020307090A0B46
:10BA90000E0F101112141718191A1B1F2021220043
:10BAA00049A3001105A400110000000002000000DD
:10BAB000EAB900110000000031B1001100000000DF
:08BAC00002000000E8B90011CA
:020000041FFFDC
:1000000000000000053D001128B8001124B80011BF
:100010009C5BFF1F000000000000000000000000CB
:1000200000000000000000000000000000000000D0
:1000300000000000000000000000000000000000C0
:1000400000000000000000000000000000000000B0
:1000500000000000000000000000000000000000A0
:100060000000000000000000000000000000000090
:100070000000000000000000000000000000000080
:100080000000000000000000000000000000000070
:100090000000000000000000000000000000000060
:1000A0000000000000000000000000000000000050
:1000B0000000000000000000000000000000000040
:1000C0000000000000000000000000000000000030
:1000D0000000000000000000000000000000000020
:1000E0000000000000000000000000000000000010
:1000F0000000000000000000000000000000000000
:1001000000000000000000000000000000000000EF
:1001100000000000000000000000000000000000DF
:1001200000000000000000000000000000000000CF
:1001300000000000000000000000000000000000BF
:1001400000000000000000000000000000000000AF
:10015000000000000000000000000000000000009F
:10016000000000000000000000000000000000008F
:10017000000000000000000000000000000000007F
:10018000000000000000000000000000000000006F
:100190006D2DFF1FCD2BFF1FC16601000000000069
:1001A000000000000000000000000000000000004F
:1001B000000000000000000000000000000000003F
:1001C000000000000000000000000000000000002F
:1001D000000000000000000000000000000000001F
:1001E000000000000000000000000000000000000F
:1001F00000000000000000000000000000000000FF
:1002000000000000000000000000000000000000EE
:1002100000000000000000000000000000000000DE
:1002200000000000000000000000000000000000CE
:1002300000000000000000000000000000000000BE
:1002400000000000000000000000000000000000AE
:10025000000000000000000000000000000000009E
:10026000000000000000000000000000000000008E
:10027000000000000000000000000000000000007E
:10028000000000000000000000000000000000006E
:10029000000000000000000000000000000000005E
:1002A000000000000000000000000000000000004E
:1002B000000000000000000000000000000000003E
:1002C000000000000000000000000000000000002E
:1002D000000000000000000000000000000000001E
:1002E000000000000000000000000000000000000E
:1002F00000000000000000000000000000000000FE
:1003000000000000000000000000000000000000ED
:1003100000000000000000000000000000000000DD
:1003200000000000000000000000000000000000CD
:1003300000000000000000000000000000000000BD
:1003400000000000000000000000000000000000AD
:10035000000000000000000000000000000000009D
:10036000000000000000000000000000000000008D
:100370007DB100110000000000000000000000003E
:10038000000000000000000000000000000000006D
:10039000000000000000000000000000000000005D
:1003A000000000000000000000000000591AFF1FBC
:1003B000000000000000000000000000000000003D
:1003C000000000000000000000000000000000002D
:1003D000000000000000000000000000000000001D
:1003E000000000000000000000000000000000000D
:1003F00000000000000000000000000000000000FD
:081838007069FF1F4118FF1F3A
:10184000024981F3088801F0B7FF00007069FF1FAB
:1018500010B501F0E1FF072804D0122808D00228B3
:1018600008D010BD044A0420136B01331363F8E75A
:101870000220F6E71420F4E7585FFF1FF8B50700D1
:101880000C0026002500503630785135002804D150
:101890000300287058342370F8BD2978CA00481E08
:1018A0008141A3183800A25C5B68C9B2FFF7D0FF82
:1018B00000280DD12B78DA00A218013350602B706C
:1018C0003378044A013B3370136A01331362D8E75B
:1018D0000123DFE7585FFF1F5C234343074910B52F
:1018E000C9180B0058331B78012B05D1FFF7C6FF31
:1018F000034A936A0133936210BDC0468C5FFF1F99
:10190000585FFF1F10B501F0C7FE064A0121130002
:1019100010CB4942D967044B136002F0BDF8200098
:1019200010BDC04600E100E01000100010B504003A
:1019300001F0B2FE024B1C6002F0AEF810BDC046D2
:1019400000E100E0431E5A425341A022F0B5D2010B
:101950005B421340154D164A40019B182A18127E0F
:101960008BB00191002A1BD01A000832D46F0022DC
:10197000E6B206AFE4B294420EDC2818C369002B2D
:1019800008D0019902AA117106AA049202AA16733C
:1019900003A898470BB0F0BD1978B9540132EAE7B3
:1019A0001A7D1A7806AB01261A70E6E71862FF1F47
:1019B00000400040F0B5254B04004001C25C85B0FA
:1019C000002A2BD01A18117E002927D0917E0029D9
:1019D00024D01179022921D11689D788D168F51B25
:1019E000ADB22A1C102D00D9102292B2BE4217D1DE
:1019F0001818012303710023C269C38003819A422E
:101A000006D06846032103730171029301A8904731
:101A10000820002C00D0192001F08EF805B0F0BD90
:101A2000013C65426C41A0256442ED012C40084D0B
:101A30001B186419074D0633013A92B2AA42EDD041
:101A40001888461C1E80085C2070F5E71862FF1F8E
:101A500000400040FFFF00000F220E4B10B59868B9
:101A6000104002380A280BD801F0F0FD0D0A0B0ACD
:101A70000A110A0A0A0A060002210020FFF762FF83
:101A800010BD0121F9E70020FFF794FFF8E7DB6FB5
:101A9000F6E7C046004000400F220E4B10B5986894
:101AA000104002380A280BD801F0D0FD0E0A0B0AAC
:101AB0000A120A0A0A0A060002210120FFF742FF61
:101AC00010BD01210800F9E70120FFF773FFF7E7D8
:101AD000DB6FF5E700900040564B70B51B68012B9B
:101AE00003D1554A936D0133936501F015FF534BB4
:101AF000534A1860534B544C1A600123534A1360E5
:101B0000534A13602378002B06D0062251495248CD
:101B100001F042FE00232370504A514B10681B789D
:101B2000C1B2002B0ED14F4CC0B223785BB2002B58
:101B30004FDB237824785BB264B21B0424021B19A8
:101B40001B1813600B1C50294ED95023464A474995
:101B50001078DBB2FF2202284BD10868444C454D77
:101B6000267890432A78964254D9227824782E7881
:101B7000023B5D10A31B6B435201D31A10335B1160
:101B80001843086001F080FF031F012B45D83A4B32
:101B90001B78002B06D0394B1B78002B02D000207D
:101BA00001F022FFA122364B92009978354B4A432F
:101BB0001B689B18832292009B181B78033B012B08
:101BC00003D8AF20400001F08FFD01222E4BDA82B6
:101BD00070BD237824785BB264B2FF33FF341B04FA
:101BE00024021B190138ABE7CAB2022AAED2022383
:101BF000ACE70868254C264D267890432A78964213
:101C000008D9227824782D78023B5B10641B63434B
:101C10005201B2E72378DBB2B2E70228D5D11D4BDF
:101C20001B78013B022B03D91B4B1B78022BCCD119
:101C30006C20C8E79809FF1FFC0FFF1F905EFF1F75
:101C4000FF3F000014100340945EFF1F0C10034080
:101C500000100340D50BFF1F7211FF1FB40003409B
:101C60008C09FF1F680AFF1F490AFF1F94000340E9
:101C7000460AFF1F470AFF1FF908FF1F2209FF1F1F
:101C8000300DFF1F3409FF1FBC0BFF1F440AFF1F4D
:101C9000450AFF1F1C09FF1F2309FF1F10B501F094
:101CA0001BFE0022014B1A8010BDC0468C5EFF1F38
:101CB00070B5244D2B68002B28D001F025FE2B6831
:101CC000D8402B680400002B27D001F0A5FE2B681C
:101CD000D8401D4B1D4A9978A1239B004B431268A5
:101CE000D118D25C91239B00002A20D0CA5801321F
:101CF000CA50174B17491B680868834214D3D23B5C
:101D0000181A012A1AD0144B186070BD01F0FCFD9E
:101D1000124B196801F0C8FED3E701F07DFE0F4BAE
:101D2000196801F0C1FED4E70D495B18E8E7CA5015
:101D30000C4B1B68DB68E418201AE4E7F530FF3031
:101D4000E1E7C0461C08FF1F300DFF1F3409FF1FCD
:101D50009C09FF1F905EFF1FA009FF1F1808FF1FAF
:101D60002DFF3F00985EFF1F70B504000D0028296D
:101D700016D10300A433C2881B889B1A0B4A9BB25E
:101D800093420DD906006A3605223100653001F014
:101D90006BFE002804D13100200001F0DDFD70BD94
:101DA0002900200001F058FEF9E7C046FE7F000040
:101DB000F8B50500012001F0DFFC134CA36AA26A0C
:101DC0009342FBD1114E336001F08EFD10490300A8
:101DD00008601048426894460F4A17680022BC45C4
:101DE00001D24268BA1A0D4802603268AD18A422C6
:101DF000E562606A520302436262094A1278002A6D
:101E000001D00F3B0B60F8BD00F00040340AFF1F0B
:101E1000E408FF1F28100040180AFF1F1C0AFF1FBC
:101E20001C09FF1F70B580241025E405A3682B430F
:101E3000A36001F041FDA368AB43A36070BD000047
:101E4000F7B5160080221C001023D205019191687D
:101E500005000B43936000225A4BD7301A6001F003
:101E6000FBFC9D232A002F009B00EB58CA32012166
:101E70000092FC37002B01D00021009A386801F055
:101E8000DBFC2900009BCB311A784F4BD3351A600D
:101E90004B780A781B0213438A7812041A43CB78D2
:101EA0001B061343494A1BBA13604B790A791B027C
:101EB00013438A7912041A43CB7931001B0613436A
:101EC000434A1BBA13606B782A781B021343AA7823
:101ED00012041A43EB781B0613433E4A1BBA1360E5
:101EE000019A330213433C4A13603C4B22001B1BF4
:101EF0009C4603293DDCB3089A0013005142B21AF4
:101F0000032A46D1354AE018511A827840781204E3
:101F100000020243E05C043302430A600022FF2B0C
:101F20004BDDF0222E4B12011A600F222D4B1A604E
:101F30002D4A1368002BFCD00023224A2749136046
:101F4000091B321D0B191B68043A180A23706070B4
:101F5000180C1B0EA070E3700434002AF2DC8022FF
:101F600010213B68D20501333B6093688B4393603B
:101F7000F7BD6346D578981893782D061B042B433C
:101F8000157804392B43557804322D022B43036016
:101F9000AFE7022A0AD1114AE05C511AE2185278DE
:101FA000120202430A6004339BB2B7E7012AB5D19B
:101FB0000A4A521AE15C1160F5E7084959180A60AB
:101FC0000433ACE7000004403C0004403800044007
:101FD00034000440300004400C0004400001044080
:101FE000040004401000044014000440F7B515003C
:101FF00080221C001023D2050091916807000B433A
:1020000093600023654AD730136001F025FC9D23BF
:102010003E009B00F9583B00CA363200FC330029D1
:1020200000D07FE0586801F007FC390032785C4B43
:10203000CB311A604B780A781B0213438A78AC467E
:1020400012041A43CB78281D1B061343554A1BBAAA
:1020500013604B790A791B0213438A7912041A43DD
:10206000CB791B061343504A1BBA13604B7A0A7A8A
:102070001B0213438A7A12041A43CB7A21001B06EF
:1020800013434A4A1BBA1360009A2B021343484A6F
:1020900013602200474B1B1B0093009BCE785B18FC
:1020A00001938B7836061B0433430E780438334390
:1020B0004E78043136023343019E33600328ECDC52
:1020C0000321A808431C9B002940800003292BD131
:1020D0003849E5185E18A9786D78E35C09042D028B
:1020E000294319433160030008330021FF2B2DDD04
:1020F000314B324919600F21314B196001232749B7
:102100000B60304B19680029FCD006211B680B407E
:10211000042B20D080220020D20593680A318B4303
:102120009360FEBD01217DE7022908D121495D1898
:10213000E1184978E35C090219432960D3E70129D2
:10214000D3D11C495918E35C0B60CCE71948181827
:1021500001600433CAE7002310490B606346002B7B
:102160000CDC3B00FC335A68102101325A6080229B
:10217000D205936801208B439360D2E7009B9B18A4
:102180001B68190A13705170190C1B0ED3700423AD
:102190005B4291709C440432E0E7C046000004407A
:1021A0003C00044038000440340004403000044047
:1021B0000C0004400001044004000440080F00002B
:1021C000100004401400044010B5002901D001F0B3
:1021D000EBFA10BDF7B5604B01919978A1239B00F4
:1021E0004B435E4A060014681022E418D6235B00B5
:1021F000E0583623FF33E35C00279343222B41D181
:10220000574B0F3A1A600760012501F03DFA019B18
:102210001880E8235B00E35C002B01D0B34258DD5B
:102220000023504FFB70AD33FF33E3581A68002A88
:1022300003D09B88DB439B071DD03823FF33E35C2F
:10224000002B18D09B235B00E35C002B13D1D13310
:10225000FF33E35CB3420EDAA4235B00E15AE018DB
:10226000090A023101F0E8FB23000122FE33013E9E
:1022700001351A87FA70E8235B00E35C002B2AD053
:10228000A8B2FEBD03683D00002BBED0818804309B
:10229000090A023101F0D0FBD6235B00E3581F602E
:1022A000B2E72300B133BA00FF3398580137818871
:1022B0000430090A023101F0BFFBE8235B00E35C54
:1022C000BB42EEDCE822F61AED1800235200A354BC
:1022D000A6E70027F1E7200001F026FA00281FD02A
:1022E000002E1DDD7319882647190193B6002000C2
:1022F00001F06AFA5A308000201840680135818860
:102300000430090A023101F097FB200001F0FCF9CA
:10231000A3590133A351BD4202D0019B9D42E6D196
:10232000114BE35C002BABD095239B00E35C002BAF
:10233000A6D00E4BE15A0029A2D00D4AA35C9942C7
:1023400002D90133A3549BE700231A212000A35490
:1023500001F092F994E7C046300DFF1F3409FF1FCA
:1023600000140340E010FF1F5A0200007202000038
:102370005E0200000D4970B54A6E0D4CD2038B69A8
:10238000D20BA24206D80B4D0224AA4204D901F076
:1023900003FB70BD02246442E21815007E24254030
:1023A0002242F4D0A3432B438B61F0E700F00040BE
:1023B0000A200000FC1C00000B001B3B70B5040051
:1023C0003020E02B0DD81300E025493BFF3B9BB2AA
:1023D000ED00AB4205D8034B200019825A8201F070
:1023E0009BF970BD8410FF1FD722044B92009B58AD
:1023F00010B5002B00D0984710BDC0460000FF1F4D
:1024000010B501F0ADF8FFF7EFFF2749274BCA6D74
:10241000274C1A4084235B001343CB65254B1B6874
:10242000186A01F0A9F9244B244A1A60244B254A62
:102430001A60A022244B52001A60244B187801F035
:1024400083FA2000224901F08FF90023A3600233B0
:10245000A360204B2049236003232048A36001F0A0
:1024600083F910221E4BFF201A60802252031A604B
:10247000802292031A60802212041A6001F0B4FADA
:10248000012001F0D1FAFA20400001F07DFA582035
:1024900001F02AF9134801F0AFF9012001F01CF90D
:1024A000072001F011FB10BD00F0004000FEFEFF10
:1024B00014100040985EFF1F000003400180063D9D
:1024C000BC00034034080000A40003404A0AFF1F78
:1024D00071020000C3090000FFFF3F002810004008
:1024E00000E100E030750000674E336888331B68F8
:1024F00083F3088801F0E8F9644A6549136800200D
:102500000B401360634B644A1B68934200D1A6E002
:1025100001F0D2FA0221614A13688B431360FFF77E
:102520006FFF5F4B5F4C1878C0B201F055F9002384
:10253000A3600233A3605C4B0120236001F01CF90F
:102540000323A36001F0B8F8040001F0E5F90500E9
:1025500001F0B2F8554B186001F026FA544B196897
:10256000621A531EA14200D213008022D20393426A
:1025700001D39B029B0A3268D16AC90700D471E07B
:102580004C491C0C09689BB24C4359432402090A6C
:10259000641803264849FC3293680A6847489B1A26
:1025A000474A0768126847499B18474A9A183340B8
:1025B0009208DB190A600360042B03D9013233400F
:1025C0000A6003600E684149A619300001F06CFAF8
:1025D0003F4F3E493B68C3183B603000019301F018
:1025E00003F93C4E3068081838493060884205D9F4
:1025F000019B01333B6001F0F7F8316001F07CF999
:10260000354B1B78002B0DD001F086F9334B621B44
:10261000196812188A4232D24919091B091A30481E
:1026200001F0A2F82F4E337A002B0ED001F074F98E
:10263000621BF1681218914224D94919091B091A21
:10264000294801F091F800233372284B83F308885E
:1026500001F02AF8002001F02FFA01F08DF901F0C5
:102660002BFA5CE7DC0199000234641A5900641A01
:1026700009214B438033CB40A408E41889E7FA21B1
:102680008900CCE71A49DBE7985EFF1F1CF0004089
:10269000FFFFC1FF0C0AFF1FB641210310000040DD
:1026A000490AFF1F14100040C3090000100AFF1F51
:1026B000340AFF1F380AFF1F200AFF1F280AFF1FC6
:1026C0001C0AFF1F240AFF1FC4090000710200003A
:1026D0006008FF1F2C0AFF1F1C09FF1FE408FF1FD3
:1026E00000100040740BFF1F3C1000400000002051
:1026F000DC050000A022054B92009B5810B5002B72
:1027000001D0984710BD01F01FF8FBE70000FF1F44
:10271000A122054B92009B5810B5002B01D0984781
:1027200010BD01F011F8FBE70000FF1FA222054BCE
:1027300092009B5810B5002B01D0984710BD01F0B6
:1027400003F8FBE70000FF1FA322054B92009B58F4
:1027500010B5002B01D0984710BD00F0F5FFFBE746
:102760000000FF1FA422054B92009B5810B5002BC0
:1027700001D0984710BD00F0E7FFFBE70000FF1F06
:1027800070B501F0C9F84F4B186000F0D5FF040098
:10279000C30702D401F088F870BD00224A4B1A60CA
:1027A0004A4B18780138042829D800F04FFF03203D
:1027B000181C2400200001F057F80128ECD0444CEC
:1027C0002378042B6ED101F0CFF80028E4D001F07B
:1027D0002BF8582000F088FF02232370DCE720004C
:1027E00000F0BAFFE9E7200001F02EF8E5E720004D
:1027F00001F09AF8E1E7200000F0C6FFDDE701F004
:1028000043F90500012808D1324B1B78053B012B09
:1028100003D82000FFF76EFFD1E72D4B1B78022B6A
:1028200001D0052B20D1022D28D12B4B9B7BAB4314
:102830001CD12000FFF76CFF264B18780128BED171
:102840006405BCD4244925224B7B034205D1233A9D
:1028500013405A42534126331A000B7D9342AED99E
:10286000322001F0B9F8AAE7022D07D1194B1B78E5
:10287000052B11D12000FFF759FFDDE7012D0BD10A
:10288000012B03D12000FFF75FFF98E7062B03D150
:102890002000FFF767FF92E7200000F055FF022DB0
:1028A0008DD1C9E7032B04D10C4B987C01F044F87F
:1028B00072E7072B00D06FE7094B987B01F0A4F873
:1028C0006AE7C0469C09FF1F9809FF1F9009FF1F78
:1028D0002309FF1F1C09FF1FA60BFF1FBC0BFF1FB7
:1028E000D40BFF1F10B500F099FE10BDF7B50B0C0F
:1028F000FF270122009300233C001E001D00944688
:10290000019089B262469A4010000840184136187A
:10291000B6B2FF2F02D1012E00D19FB20098024023
:102920001A41AD18ADB2FF2C02D1012D00D19CB2DD
:102930000133102BE6D10320012E07D1012D04D144
:10294000019B2401E4191C700138FEBD102EFCD13E
:102950000238102DF9D00230F7E700008023F7B5D8
:102960009C46264B264F01932649274A274D284C43
:10297000284B02281AD1604638600868264E30403D
:10298000802636033043086001990978002909D16F
:102990001660224A2A60224A2260E0221968914386
:1029A000A03A1BE08021C9021160F2E766463E6052
:1029B0000F68194E3E408027FF023E430E6001998A
:1029C000097800290DD1176001280ED1154A2A6017
:1029D000154A2260E02219689143C03A0A431A60FE
:1029E000F7BD802189021160EEE7E0210F4A024322
:1029F0002A600F4A22601A688A43F0E74B0AFF1FD9
:102A0000E0000340D8000340900003400000034072
:102A10005000034040000340FFFFE3FF0280063DFB
:102A2000804508220180063D8066082200800698C5
:102A300080550822F8B51E4B80261A680020140025
:102A40003440324232D11A681A4F32431A6001229E
:102A50003B68063093433B6000F08EFE0122164D2A
:102A60002B681E432E603B680A2613433B60802779
:102A7000BF00124B1B683B4211D1013EF6B2FF2E44
:102A800009D17E220E4B1C682B68E40B1440934343
:102A900023432B6005E0082000F06EFEE9E7002EDE
:102AA000EFD180222B68600893432B60F8BDC046AD
:102AB000C4F000405CF0004018F0004068F00040B6
:102AC00060F0004010B500F0BFFF01215820034A1C
:102AD00000F0FAFDFFF7AEFF10BDC046600AFF1F11
:102AE00010B578220021034800F086FF00F064FF53
:102AF000002010BDA061FF1F70B5040000F0CCFDE8
:102B000000230C200B4A010059438D18515C002909
:102B10000DD0A14208D1012300246B7000F0ECFD20
:102B200000F0BAFF200070BD01330A2BEBD1122454
:102B3000F6E7C046A061FF1F70B5040000F0ACFDD1
:102B4000002319001D000D4A1078002806D0A0426D
:102B50000CD1557001310C320A29F5D1002B0AD164
:102B600000F02AFF00F098FF002070BD5078461E4C
:102B7000B0411B18EEE700F0BFFDF3E7A061FF1FB7
:102B8000F7B504000C20002384460E4D01926746E1
:102B90005F43E85D7E19A04212D000280BD10A4B9A
:102BA0009C4662461B7808331370019B70707C55FD
:102BB0007160B360FEBD01330A2BE8D10320F9E751
:102BC0000720F7E7A061FF1F9C61FF1F8020F8B579
:102BD000484BC0051B68C1248360474BFF251A681A
:102BE000012313434361454BA4001A68444B402121
:102BF0001A60444B1A68444B1A60444B1A59AA4352
:102C00001A51C52292009E58AE43314380269950F6
:102C10009F583F49F6010F403E439E509E588027E3
:102C20003602360A3043985080201A5900020A4072
:102C300002431A5104341A59364E3F04324080265A
:102C40003A431A511A5936061202120A32431A51DD
:102C500008341A5980260A4002431A51C3229200AE
:102C60009F58B446AF4337439F509F58294E0F405B
:102C700007439F509F5837408026360437438026AD
:102C80009F509F5836063F023F0A37439F50C0224D
:102C90001F59AF433A431A511A591202120A1643E6
:102CA000C6221E5192009C58AC4365462C439C5052
:102CB0009C5800250C4020439850C72080001A588B
:102CC000154C1140C02212020A431A50134B1B78B4
:102CD000DB08AB4201DC0020F8BD2378002B06D0D6
:102CE000A368002B00D0984701350C34EEE7122082
:102CF000F2E7C046C83DFF1FC43DFF1FB0F00040D3
:102D00009861FF1FB4F000409461FF1F00E100E0F4
:102D1000FF00FFFFFFFF00FFA061FF1F9C61FF1F7F
:102D2000030010B51F2809D80722002013400724EC
:102D300004490A78A24313430B7010BD00230620F8
:102D4000F5E7C0469C61FF1F054B06491B780A68E2
:102D500005485B0702401B0B134300200B607047C4
:102D60009C61FF1F1CF00040FFFFC1FF70B50C25E8
:102D7000FFF7EAFF0A4B1C780A4BE4086543ED189D
:102D8000002C01D1200070BD2B78002B06D06B6881
:102D9000002B00D09847013C0C3DF1E71220F2E7F0
:102DA0009C61FF1F9461FF1F1FB5002102220B00D1
:102DB00001910091052000F05FFD02230B490A6894
:102DC0001A42FCD120230393039B5A1E0392002B2B
:102DD000FAD1074A1368002BFCDA0B246C4420005C
:102DE000012100F011FD207804B010BD90C8004012
:102DF00000C8004013B504000A4B0193019B002B4F
:102E000001D1112016BDFFF7CFFF2300034004427C
:102E100005D0052000F0B0FC019B013BEDE7180058
:102E2000F0E7C046FFFFFF0707B500F035FC802242
:102E30000821D205936A0191002B01D107399162D3
:102E400002210C4A11600199481E01900029FAD113
:102E500003311160053101910199481E019000294B
:102E6000FAD11160002B02D18022D205936200F0CA
:102E700013FE07BD00C00040F0B52D4C89B023788B
:102E8000002B4FD1FEF73EFD02232A4F03903A68F4
:102E90001A42FCD120230693069B5A1E0692002B51
:102EA000FAD1254E3368002BFCDA0120FFF7A2FF90
:102EB000011E02D0112009B0F0BD030003220190D1
:102EC000009005AD9F2000F0D7FC0321280000F002
:102ED0009BFC02233A681A42FCD120230793079BEC
:102EE0005A1E0792002BFAD13368002BFCDA01201E
:102EF000FFF780FF0028DDD10398FEF717FDAA78C1
:102F00006B7811041B020B4329780B436360130099
:102F1000113B0A49052B07D801239340A3600B609E
:102F2000012323700020C6E780231B03F6E7C04679
:102F3000B03DFF1F90C8004000C800409808FF1F28
:102F40001E4B30B55A6818781D4B85B0D3185942BE
:102F50004B4101210093002300F096FC194B1A4AC3
:102F600002259A6300221A6510325A658022C42114
:102F70009D65164B1648D202DA6789004258154BF8
:102F800080241A4080231B041343435064234120B0
:102F90000393E40500F006FA402000F003FA6562AE
:102FA000039D6B1E0393002DFAD103236362FFF789
:102FB0003BFFA562FFF760FF05B030BDBC3DFF1FC2
:102FC00095FFFEF700C80040050001FF04E100E0A6
:102FD00000E100E0FFFF00FFF0B585B00700FEF75D
:102FE00091FC022305002D4C22681A42FCD12023BB
:102FF0000093009B5A1E0092002BFAD1284E336892
:10300000002BFCDA0120FFF7F5FE002803D0112485
:10301000200005B0F0BD234B2360022322681A4232
:10302000FCD120230193019B5A1E0192002BFAD15F
:103030003368002BFCDA0120FFF7DCFE0028E6D124
:10304000194B1F60022322681A42FCD120230293ED
:10305000029B5A1E0292002BFAD13368002BFCDA35
:103060000120FFF7C7FE0028D1D1104B23600223B7
:1030700022681A42FCD120230393039B5A1E039219
:10308000002BFAD13368002BFCDA0120FFF7B2FEE7
:10309000041EBCD12800FEF749FCB9E790C80040E7
:1030A00000C8004001000006A8C8004001800001DF
:1030B00010B50020FFF790FF10BD000010B5064BC3
:1030C00018705960FFF73CFF00211320034AFFF7F7
:1030D00057FD002010BDC046BC3DFF1F412FFF1F04
:1030E000F0B5040085B003920291FEF70BFC882234
:1030F00063035B0B52051A438023DB059D6A802323
:10310000274F0092BA68002601901B039A420CD9FF
:10311000F82326001B041E401C4206D08022214BAF
:1031200052025E6219680A431A60002D0BD100F04A
:10313000B3FA02221C4B1A608023DB055A62013A63
:103140009A6200F0A9FC0023039A934220D1002D3B
:103150000AD100F0A1FA144B03221D608023DB0585
:103160005A629D6200F098FC8023BA681B039A4261
:1031700008D9002E06D000220A4B0C495A621A6860
:103180000A401A600198FEF7D1FB002005B0F0BD9F
:10319000009A0299D2181278CA540133D4E7C04673
:1031A000B03DFF1F00C8004000C00040FFFFFEFF11
:1031B000F0B587B0029103920400FEF7A3FB0190E3
:1031C00000F06AFA802302250122234EDB053560D8
:1031D0005D629A6200F060FC204F3B682B42FCD19C
:1031E00020230493049B5A1E0492002BFAD11C4DF9
:1031F0002B68002BFCDA0120FFF7FCFD002802D031
:10320000112007B0F0BD2000039A029900F034FCB1
:10321000022304003A681A42FCD120230593059B3F
:103220005A1E0592002BFAD12B68002BFCDA0120E4
:10323000FFF7E0FD051EE3D100F02EFA8023032204
:10324000DB0535605A629D6200F026FC0198FEF7AE
:103250006DFBE0B2D5E7C04600C0004090C800401A
:1032600000C80040F0B5802489B00600FEF74AFB94
:10327000E405A36A02250393029000F00DFA0123EE
:10328000304F3D606562A36200F006FC2E4C23685F
:103290002B42FCD120230593059B5A1E0592002B3F
:1032A000FAD12A4D2B68002BFCDA0120FFF7A2FD92
:1032B000002803D01124200009B0F0BD244B236066
:1032C000022322681A42FCD120230693069B5A1E31
:1032D0000692002BFAD12B68002BFCDA0120FFF7B5
:1032E00089FD021EE6D11B4B03211E6003000190E5
:1032F0000090202000F0C0FA022322681A42FCD17C
:1033000020230793079B5A1E0792002BFAD12B68A4
:10331000002BFCDA0320FFF76DFD041ECAD100F07C
:10332000BBF980230322DB053C605A629C6200F0FB
:10333000B3FB039B002B01D1FFF776FD0298FEF74C
:10334000F5FAB8E700C0004090C8004000C800404F
:103350000100000694C8004007B500020191042254
:10336000000A01A9FFF724FF0EBD000073B5050098
:1033700005240B4AA3005B429B1819686B46DE1DAF
:103380003000FFF7B3FA022804D133782B55013C03
:10339000EFD276BD052CFCD00128FAD10230F8E737
:1033A000140900111F2807D8012380228340D20569
:1033B00091680B43936070473F2808D8012380220F
:1033C00020388340D20551690B435361F3E75F28EE
:1033D000F1D80123802240388340D205116A0B4383
:1033E0001362E8E71F2807D8012280218240C9051F
:1033F0008B6893438B6070473F2808D80122802157
:1034000020388240C9054B6993434B61F3E75F283D
:10341000F1D80122802140388240C9050B6A9343CC
:103420000B62E8E71F2810D880230200DB05153A5D
:103430001968012A06D820229143196019680A43A5
:103440001A60704701228240F6E73F2811D8802396
:103450000200DB05353AD968032A06D810229143C9
:10346000D960D9680A43DA60EBE70122203882404C
:10347000F5E75F28E5D842238022181A413B8340B4
:10348000D205516A99435162516A0B435362D8E79E
:1034900010B50400012813D1A022184992050B6829
:1034A0005B015B0913430B60154B164A1968114009
:1034B000154A0A431A60402219680A431A6010BD6F
:1034C0000028FCD101000A2000F0E6F921000B20C1
:1034D00000F0E2F9C0220A4B920019680A43402129
:1034E0001A601A688A431A60B022044912060B68EF
:1034F0005B015B0913430B60E1E7C04614F0004039
:103500001CF000407F00FEFF80FD010072B6074AFC
:103510001368013313600422054B1A600023054A27
:1035200013608022D2055360FEE7C0467808FF1F73
:10353000C0F00040C4F0004005490B68002B05D1E5
:10354000044A0A6004490A60044A13607047C0468E
:10355000140AFF1F841E0000380AFF1FC4F0004039
:103560000023034A1360034A1360034A1360704741
:1035700054F0004040F1004044F10040002310B5F9
:10358000184C8AB0009301932378012B27D0694609
:10359000012000F019FA002817D1009B124902936C
:1035A000019B06AA0393114B02A81B680493104BBE
:1035B0001B68059300F080F910220E4906A800F060
:1035C00053FA002804D1FF23237000200AB010BD55
:1035D0000123094A074902A8237000F06DF9012070
:1035E000F4E7C0469C5EFF1F102900110829001156
:1035F0000C29001120290011A05EFF1F13B5012422
:103600006946012000F0E0F9034B00940193FFF7B5
:10361000B5FF200016BDC046BB0B000010B5FFF77C
:103620009FFFFFF7EBFF002802D0024B984710BD29
:10363000FEE7C046E1A2000002B471464908490015
:10364000095649008E4402BC7047C04602B4714618
:1036500049084900095C49008E4402BC7047C046D5
:1036600003B47146490840004900095A49008E4494
:1036700003BC70470000000001B40248844601BC4E
:10368000604700BF53B9000001B40248844601BC42
:10369000604700BFCD0C010001B40248844601BC64
:1036A000604700BF75A9000001B40248844601BC10
:1036B000604700BF7997000001B40248844601BC0E
:1036C000604700BF156B010001B40248844601BC8D
:1036D000604700BF0167010001B40248844601BC95
:1036E000604700BFE512010001B40248844601BCF6
:1036F000604700BF7912010001B40248844601BC52
:10370000604700BF21A9000001B40248844601BC03
:10371000604700BF5976010001B40248844601BCED
:10372000604700BF116E000001B40248844601BC2E
:10373000604700BF71B0000001B40248844601BC7C
:10374000604700BFBD0B010001B40248844601BCC4
:10375000604700BFE917010001B40248844601BC7C
:10376000604700BF0934010001B40248844601BC2F
:10377000604700BF2D6C010001B40248844601BCC3
:10378000604700BF0189000001B40248844601BCC3
:10379000604700BFF935010001B40248844601BC0E
:1037A000604700BFE94C010001B40248844601BCF7
:1037B000604700BFE9D4000001B40248844601BC60
:1037C000604700BF85B1001101B40248844601BCC6
:1037D000604700BFD9B0000001B40248844601BC74
:1037E000604700BF8914010001B40248844601BC4F
:1037F000604700BF090E000001B40248844601BCC6
:10380000604700BF8D11010001B40248844601BC2D
:10381000604700BF3D71010001B40248844601BC0D
:10382000604700BFE927000001B40248844601BC9C
:10383000604700BF6DF6000001B40248844601BC39
:10384000604700BF2144000001B40248844601BC27
:10385000604700BF0534010001B40248844601BC42
:10386000604700BF8944000001B40248844601BC9F
:10387000604700BF0134010001B40248844601BC26
:10388000604700BF496D010001B40248844601BC95
:10389000604700BFC56D010001B40248844601BC09
:1038A000604700BF099E001101B40248844601BC74
:1038B000604700BFDD0A010001B40248844601BC34
:1038C000604700BFDD3F000001B40248844601BCF0
:1038D000604700BFC9A9000001B40248844601BC8A
:1038E000604700BF8D82000001B40248844601BCDD
:1038F000604700BFBD5C010001B40248844601BCC2
:10390000604700BFD544010001B40248844601BCB1
:10391000604700BFE90B010001B40248844601BCC6
:10392000604700BFC95C010001B40248844601BC85
:10393000604700BFF535010001B40248844601BC70
:10394000604700BF4DF9000001B40248844601BC45
:10395000604700BFEDA5000001B40248844601BCE9
:10396000604700BF85C1000001B40248844601BC25
:10397000604700BF01D7000001B40248844601BC83
:10398000604700BF8552010001B40248844601BC73
:10399000604700BF8512010001B40248844601BCA3
:1039A000604700BFD1AE000001B40248844601BCAC
:1039B000604700BFC166010001B40248844601BCF3
:1039C000604700BFADAE000001B40248844601BCB0
:1039D000604700BFE1AC000001B40248844601BC6E
:1039E000604700BF6137010001B40248844601BC52
:1039F000604700BFED6B010001B40248844601BC82
:103A0000604700BFB70E000001B40248844601BC05
:103A1000604700BFC1F7000001B40248844601BC02
:103A2000604700BF6D0B010001B40248844601BC31
:103A3000604700BF6911010001B40248844601BC1F
:103A4000604700BFC115010001B40248844601BCB3
:103A5000604700BFED68010001B40248844601BC24
:103A6000604700BF51B8000001B40248844601BC61
:103A7000604700BFCD4C010001B40248844601BC40
:103A8000604700BF9573010001B40248844601BC41
:103A9000604700BFDD0C010001B40248844601BC50
:103AA000604700BF9DA9000001B40248844601BCE4
:103AB000604700BF090E000001B40248844601BC03
:103AC000604700BF016C010001B40248844601BC9C
:083AD000604700BFF90D010081
:103AD80002000000E6B900110100000018B800114A
:103AE80002000000E2B9001101000000183BFF1FAE
:103AF8000200000020B80011010000001C5CFF1F3C
:103B080002000000E0B9001103000000905BFF1FF5
:103B18001200000002000000E6B9001101000000D8
:103B280060B8001102000000E2B9001101000000B5
:103B38005DB80011020000006AB80011030000001F
:103B4800CB5BFF1F02000000E0B90011030000007A
:103B5800E05BFF1F02000000E2B900110100000055
:103B68005CB800110200000068B8001103000000F2
:103B7800A15BFF1F02000000E0B900110300000074
:103B8800C25BFF1F02000000E6B90011010000003F
:103B9800A0B8001102000000E2B900110100000005
:103BA800613CFF1F02000000B2B8001101000000D4
:103BB8009BB8001102000000E2B9001101000000EA
:103BC800603CFF1F02000000B0B8001101000000B7
:103BD800E85BFF1F02000000E2B9001101000000CD
:103BE8005F3CFF1F02000000AEB80011010000009A
:103BF8008BB8001102000000E2B9001101000000BA
:103C08005E3CFF1F02000000ACB80011010000007C
:103C180086B8001102000000E2B90011010000009E
:103C28005D3CFF1F02000000AAB80011010000005F
:103C380081B8001102000000E2B900110100000083
:103C48005C3CFF1F02000000A8B800110100000042
:103C58007CB800110202020202020000000000000B
:103C68000D0C0000E14A0011A54A0011F4B800113A
:103C780090011D0018001800FFFF0701020304054A
:103C8800060201060000000000000000000000001D
:103C9800000000000000000000000000000000001C
:103CA8000300000002000000E6B900110100000056
:103CB80014B9001102000000E2B90011010000006F
:103CC8001C3DFF1F020000001EB90011010000008A
:103CD800165CFF1F02000000E0B90011030000009D
:103CE800805EFF1F02000000E2B900110100000021
:103CF8001C3DFF1F020000001CB90011010000005C
:103D0800185CFF1F02000000E0B90011030000006A
:103D1800785EFF1F12000000000100000000011182
:103D2800FFFF000050485936000000000000000066
:103D38000B000500F0000000B4000028002800284F
:103D48003075A000A000A000A00000080008E00155
:103D5800F0001000100010001000100010005000BB
:103D68005000500010001000D007000000000000B4
:103D78000F0001000500307507001000010081FFE9
:103D880000000000FF000000F16F0011F96D001144
:103D9800896B0011FFFF0100FF0000000D9A001160
:103DA80089970011A1960011000000000000000092
:103DB80000000800040000003B0001085902E0016F
:103DC8008821280002000000E6B900110100000067
:103DD800ACBA001102000000E2B9001101000000B5
:103DE800493EFF1F02000000DEB90011010000007B
:103DF8005862FF1F02000000E2B900110100000034
:103E0800483EFF1F02000000DCB90011010000005D
:103E1800463EFF1F02000000E2B900110100000049
:103E2800443EFF1F02000000DAB900110100000043
:103E38003C3EFF1F180018001D00900102000003FF
:103E48000202000002000000E6B9001101000000B3
:103E5800C0BA001102000000E2B900110100000020
:103E68008C3EFF1F02000000D8B9001100000000BE
:103E78000000000002000000E0B90011030000008B
:063E88007862FF1F20FF1D
:040000051FFF184180
:00000001FF
